:020000041100E9
:10300000002310B5294C0120636101F0EFF9402045
:103010000223FE21264A207401F06EFA002835D1E1
:103020000223FF21234A207C01F066FA00282DD1DB
:10303000214BA2899A4226D1E389204A93420ED19C
:103040001F4B204963612368002B05D1002903D061
:103050000C22200008F0BCFB01F03CFA10BD1A4A1B
:10306000934201D00021EEE7184B194A1B689342A6
:1030700005D9C0220421207C920001F0B7FA104B40
:1030800014496361DFE700232374EBE7CC22382087
:10309000AC219201207401F0A9FA0028F3D10E4B63
:1030A0000E4963610E4BE381CDE7C046E862FF1F26
:1030B000F462FF1FF662FF1F5959000083050000EC
:1030C00051420011A4BB0011821500002C63FF1FA8
:1030D00087130000B0BB0011ED42001198BB001136
:1030E000AAAAFFFFF7B5164B0192C318021D0020D4
:1030F000009388235B05D3181B685C1C1AD09CB214
:10310000402C18D88D781E0CAC466746CD782D0221
:103110003D43AE4206D1019800280ED110000C703C
:10312000240A4C7003249BB20733A343D218009B9C
:103130009A42DED3FEBD4432F9E71000FAE7C046FA
:10314000FC0F0000802213B503000324019189B213
:10315000520107319B18A14304305A1A88235B059A
:10316000C3181B68591C03D190429241104016BDF0
:1031700099B2402907D80B000733A343C0189042E7
:10318000ECD30020F3E74430F9E7134B134A1B68F4
:10319000126810B5FA24934201D81A00F824104B93
:1031A000E4021B689A4210D813000E4A12689A4231
:1031B0000ED3013307D1F823DB029C4203D10A4925
:1031C000054808F015FA200010BDFC24E402ECE7E5
:1031D000FE24E402F7E7C04600C0071100D0071143
:1031E00000E0071100F00711FFFFFF7FF0B59BB073
:1031F000150004900391402A00D9A0E006AB598045
:103200001A80FFF7C2FF0400042816D9002206A97D
:10321000FFF768FF052810D906AB1B88AB420CD11D
:10322000002D07D0514B2A000499C01808F018FA55
:10323000002802D101201BB0F0BD06AB1D8020008C
:103240000699FFF77FFF041E7BD1069B0793FFF7CC
:103250009CFF80235B01C618802307001B039E424E
:1032600001D3F826F60288235B05F31801931B6847
:10327000013302D0019808F0CBF93D49019808F0DC
:10328000B7F93B1D0293331D05938822029B52051B
:103290009B181B6808935A1C3CD044219AB2009199
:1032A000402A04D80320D11D814389B2009103999B
:1032B0001B0C8B4224D0402A22D80122300008A9BE
:1032C000FFF710FF021E1BD1380008A9FFF70AFF05
:1032D0000400042831D9009A059B9B1880225201D2
:1032E000B218934240D288235B05C118009A09A8FE
:1032F00008F026FA1D4B009A09A9F01808F0A8FB5F
:10330000009A029B9446634402931A4B029AFB185C
:103310009A42BAD388235B05FC18216801980139C9
:1033200008F066F9200008F073F9039A07AB5A8099
:1033300030000799FFF706FF0400002C03D100209E
:1033400079E70428FBD988235B05E018069908F083
:103350004FF90323EA1C9A4300D16BE7034B04990E
:10336000E01808F075FB65E70424ECE704000011A1
:10337000FFFFFF7FF80F0000F7B505001400402A9B
:1033800021D8002701AE71803780FFF7FEFE0428A8
:1033900016D93A003100FFF7A5FE042810D9368867
:1033A000BC420BD0BD4209D0221CB44200D9321C11
:1033B000064B92B2C118280008F0C2F930B2FEBD27
:1033C000C04300B2FBE703204042F8E704000011CD
:1033D00037B5042204000D0001A81649FFF7CCFF01
:1033E000020004280BD1019BA34208D3AB4204D0B6
:1033F000104901A80195FFF7F9FE01203EBD0E4CD2
:1034000023682000019308F003F901992000013995
:10341000019108F0EDF880235B01E418074B9C4212
:10342000EED10422034901A80195FFF7DFFE002039
:10343000E4E7C0465555000000C007110000081120
:1034400030B589B008F07CF810226946254808F0AC
:103450005FF9254B009A9A420ED1019B029A0F2BDD
:1034600033D8002101240698013B08D2002900D05E
:103470000292029B013331D10023029325E0551CB7
:10348000F2D102002100EFE710341022200004A93D
:1034900008F03EF9029B013301D1069B0293882379
:1034A00004995B05C918059B06981A03120B049131
:1034B0000592814203D02B4201D108F089F9019B8A
:1034C000013B0193019B002BDED1029B002B03D01B
:1034D000049304984168084709B030BDE025014CC9
:1034E0002D03EFE70000011150485936F7B50F4999
:1034F0000F4B0A6804001A4084235B0013430B60DF
:10350000030003271033019300252E00112008F03B
:10351000CFF9084B1B683B40AB4002351E43202DC2
:10352000F4D1019B40C4A342EED1F7BD5CF0004052
:1035300000FEFEFF64F00040802270B5AD4CAE4B43
:10354000D200002120001C6008F0A2FA2300AB4A40
:1035500088331A60AA4B1A786E23002A00D01133E0
:10356000E3620A232365A74B1878A74BA0630138B1
:10357000E361C3B2032B01D810232362A34B37228C
:103580006361C823DB00A36123008C331A60082326
:1035900036210F3AE518E16323646264E967043970
:1035A000251DE96725003B26BC352E602500C0356A
:1035B0002B602500C4352A6025000636CC352E60E8
:1035C0002500083EC8352E602500D0352960210031
:1035D000D4310B602100D8310A6021000225E0318E
:1035E0000D6025004221DC35296025001B3EE435B5
:1035F0002E602500E8352B602500EC352A6022007E
:103600000525F43215602200F032116022001831D5
:103610009032116022009432136023003C229833D0
:103620001A60AF23DB002360794B2363032805D89E
:1036300008F0DEF833023537152363609623210046
:10364000FA225B00A360E360C8332361714BFC3155
:103650009200A3640A6062626F4A704DA262732294
:10366000E2656D3A6265A2650232E5644A60022154
:10367000616696218900A166626709210022E166E0
:10368000A2676749674A684E2167E2673560032889
:1036900011D808F0ADF896089EA61023CDE70E23AA
:1036A000CBE70C23C9E720001A259C3005602000D9
:1036B0000735A03005602000A83003602300FA2001
:1036C000F8338000186023006420A43318602300BE
:1036D0005F38AC33186023000338B0331860230020
:1036E000C630B433186023000020B83318602300BC
:1036F0003825FC339D604D4D5A665D644C4D9A648F
:10370000DD619625AD001D624A4D9A675D62F53D0B
:10371000FF3D9D621E25484ADD6618675867D965DA
:103720001966DA67BE23C021444A5B00E250444B6D
:103730004900635004316250C4225200A350FA235E
:10374000E4205B000432A3500432A3503D493E4ABA
:103750003E4BD1603E49800019503E49E938FF3860
:1037600019503D49043019503C491038D1613C4949
:1037700011633C4951633C4911603C49195019009F
:103780003B48F83108603B49D16582213A4A8900BB
:103790005A501A0039490832D1671A003849B432F0
:1037A00011608821374A89005A501A0036498832F8
:1037B0001160364ADA6407F04BFE012007F058FF2B
:1037C00070BD200014259C30056020000435A03019
:1037D00070E7200010259C30056020000335A030E4
:1037E00068E720000E259C30056020000235A030DF
:1037F00060E7C0460004FF1FC465FF1FB070FF1FD5
:103800007C45FF1F4A0AFF1F3A07000080C3C90119
:103810009A02000050C300006A180000280A000045
:10382000204E000088130000F009FF1F0040001127
:1038300068100000C4090000DC05000040420F00D1
:1038400010270000FD1BFF1FFC00FF1F0000FF1FD3
:10385000252FFF1F4D32FF1FE530FF1FD91FFF1F10
:10386000F51FFF1FA121FF1F491FFF1FC528FF1FB5
:103870008D2CFF1FD918FF1FD127FF1F3925FF1FD0
:103880004525FF1F491EFF1F011FFF1FC11DFF1FF1
:10389000F7B50B0CFF270122009300233C001E000C
:1038A0001D009446019089B262469A40100008407B
:1038B00018413618B6B2FF2F02D1012E00D19FB2A7
:1038C000009802401A41AD18ADB2FF2C02D1012D73
:1038D00000D19CB20133102BE6D10320012E07D179
:1038E000012D04D1019B2401E4191C700138FEBD97
:1038F000102EFCD10238102DF9D00230F7E710B5A8
:10390000064C2378002B07D10548FFF7EFFD05484B
:10391000FFF7ECFD0123237010BDC0468465FF1F37
:103920009865FF1F8865FF1FF0B58BB00D00012360
:103930000190102936D8FFF7E2FF00231A001B4838
:10394000C15C01335218102BFAD1023B002A29D056
:10395000174B184C1F68002306A9E25C1600FA5C9E
:1039600056405E540133102BF7D102AA08F010F82C
:103970002A0002A9019807F02BFF07F049FF2368EE
:103980001B18236007F044FF63681B18636007F08F
:103990003FFFA3681B18A36007F03AFFE3681B18FA
:1039A000E360002318000BB0F0BDC0469865FF1F10
:1039B0001C44FF1F8865FF1F0223F0B50124574EEA
:1039C000574D3370574B2C701B688FB0552B10D050
:1039D000082006F0E9FA00280BD00023210000930C
:1039E0000420514A08F004F88023DB059C62FFF7AD
:1039F00027FD002006F070FD07F09AFEFFF79CFD02
:103A000007F0B6FD1F2201240021484B0EAF1A70AB
:103A1000474B1C70474B1970474B19689143163A36
:103A20000A431A60602219689143403A0A431A60B7
:103A300007F056FD07F07CFDC120FF213F4B8000C1
:103A40001A588A431A50C522920098588843BF39A1
:103A50000143995098583A4908408021C9010143CF
:103A6000802099509958C0050902090A01439950CC
:103A700080213448490107F003FD03232200324925
:103A800001940093314807F04BFF2C22304903A8E2
:103A900007F056FE03AC61782078023406F0AAFAEB
:103AA000BC42F8D10121002006F0BEFB294B2A4A76
:103AB000196803201140A022D2020A431A60802212
:103AC000196892040A431A601968244A1140802236
:103AD00092030A431A60224B224A934200D80120E3
:103AE00007F0EEFD07F00CFD07F00AFF307807F055
:103AF0005FFE2878C0B207F043FE07F011FD0A49C7
:103B0000042007F005FF06F0B3FC00F09FF800F07A
:103B10002BFE00F00BFA00200FB0F0BD4A0AFF1F89
:103B20007C45FF1F34F000403B000108480AFF1F9E
:103B3000490AFF1F680AFF1FBCF0004000E100E0D7
:103B4000FF00FFFF8045FF1F0458FF1F8055FF1F28
:103B5000C0BA001114F00040FF7FF8FFFFFF9FFF85
:103B6000B070FF1F0080FF1F70B500252849294A4B
:103B700029484D6308CA1B051B0DED188242F9D177
:103B80000022264B8B63264B08211A628022254B8C
:103B90009205DA67244BDA688A43DA60234A12789E
:103BA000012A03D09A6822490A409A600121EE2432
:103BB0002048E40002686C438A430260DA681120FE
:103BC0008A43DA6007F0B4FE112007F071FD11207E
:103BD00007F0D6FC184A200C0400642390420AD84F
:103BE000FA220023D200904205D9144B0A21C018B2
:103BF00007F016FCC3B2124A1372124BD4801B7822
:103C0000002B04D1104B1021187807F031FF70BD44
:103C1000000005408805054000060540FF01000042
:103C200000F0004004E100E03CF000404A0AFF1FC1
:103C3000FFDFFFFF00380040B70B000030F8FFFF48
:103C40000063FF1F3865FF1F2863FF1F002210B5A8
:103C50001100112007F0ECFD10BD0000F8B50023A5
:103C600001250826394F3A4C3B62E3681120AB43EB
:103C7000E360E368B343E36007F01AFD112007F047
:103C800057FE112007F00CFD402322682900134342
:103C9000236080236268DB02134380226360A36891
:103CA00007201343A360A3682A4A1340A36080231C
:103CB000A2689B0113431022A360236C93432364E7
:103CC000236C2B43236480235B003B62226B224BDB
:103CD0001A402263626B1A406263A26B1A40A263AD
:103CE000E26B1340E3631D4AE3681340E36006F0B0
:103CF0006BFA2900072006F097FA8021184A112054
:103D0000536C0B43536407F05BFCFD21154B164AC3
:103D100089005A508023C720626B5B03134363639F
:103D2000E36880003343E360E368104A1D43104BAF
:103D3000E56019581140802212020A431A5080226D
:103D400092051A600B4B5E63F8BDC04600F0004060
:103D50003CF00040FFFFDFFFEFFFEFFFFFFF7FFFC3
:103D6000003800400000FF1F693B0011FF00FFFF0B
:103D700000E100E00000054030B503A804880B20F6
:103D8000002C0ED14968074D087849780902014393
:103D90000A20A94205D1012120001980024B1B7A7B
:103DA000137030BD192A00000063FF1FF7B515001E
:103DB00008AA16884A680F4F1478527812022243D4
:103DC0000A24BA4214D10122DBB2019200962A00E1
:103DD00007F09EFA041E0BD1074B1B68002B07D07F
:103DE00068782A78000210434242504101309847D7
:103DF0002000FEBD022900008462FF1F30B50125AE
:103E000003790400BFB02B4212D00A49408806F063
:103E1000EBFD28420CD06A46074B69465B8D558006
:103E20001380064B60881B7A1371002203F0A2FEF8
:103E30003FB030BD7C62FF1FC041FF1F0063FF1F0A
:103E400010B50549054806F085FD0421044A0548DA
:103E500006F042FD10BDC0467C62FF1FFFFF000060
:103E6000ECBA0011C041FF1F10B5024804F004FD78
:103E700010BDC046FD3D0011062310B58370103300
:103E80000371443B43712A3383714433C37100236C
:103E90000222012103720E4B027041701C88817254
:103EA0004472197A0273C1729A784273DA78827313
:103EB0000322C2731A7902745A7942740C228274F2
:103EC0009A79C274DB7903751123C370152010BD74
:103ED0000063FF1F10B5142007F072FD124B14226F
:103EE0000021186007F074FD002007F051FC01204C
:103EF00007F06EFB022007F003FC032003F060FFD5
:103F0000042005F075FF052003F09EF9062003F05C
:103F10006BFE072001F0C4F8082006F0BDFC092064
:103F200000F0A2FE10BDC0468862FF1F10B507F06A
:103F300057FD012007F014FB07F0D2FB002010BD55
:103F4000094B10B50400984205D0012904D1200086
:103F5000064906F0FFFC10BD0229FCD1013904F02E
:103F600049FC0028F3D0F6E7FEFF0000AE62FF1F19
:103F700070B50D7A100004AA2C0016881022144087
:103F8000154220D1002E20D10A78022A18D14A6881
:103F9000517815780E4A09022943914205D00D4AFD
:103FA000914209D01C800A2404E014220A491A8094
:103FB00007F00EFC200070BD0C2208491A80F7E7BC
:103FC0001C800124F6E70824F4E70B24F2E7C0463E
:103FD000F3FF0000F4FF00000044FF1FC8BB001106
:103FE00010B504000749084806F0B4FC074804F07F
:103FF00083FB0020E40704D50721054A054806F0A5
:104000006BFC10BDAE62FF1FFFFF0000413F0011BF
:1040100030BB00110442FF1F00B50C4BBFB01A7833
:104020000B4901A800F0D4FB6B4680B258800028F1
:1040300009D06A46074B69461B881380064B00224D
:10404000188803F097FD3FB000BDC0468C62FF1F8B
:104050008D62FF1F5E42FF1F5E43FF1F00B50C4BCA
:10406000BFB01A780B4901A801F0C6FC6B4680B2BC
:104070005880002809D06A46074B69465B8D13803B
:10408000064B0022188803F075FD3FB000BDC04606
:10409000B662FF1FB762FF1F0442FF1F5E43FF1F90
:1040A000F7B50E00377A1C0008AB11003D001A88E6
:1040B00020231D401F423CD13378022B3BD1736833
:1040C0001F785B781B023B431E4FBB4208D01E4F3C
:1040D000BB4214D01D4DAB4221D00A252800FEBDA5
:1040E000002A2AD1142C2AD82200F06807F070FB8D
:1040F000174B1C70012CF1D9FFF7B0FFEEE7002A37
:104100001BD1202C1BD82200F06807F061FB114B5B
:1041100004211C70104B187807F0AAFCDEE7E3B20C
:104120000124009201940A00310007F0F1F8050023
:10413000D4E70825D2E70125D0E70B25CEE70D25EA
:10414000CCE7C046F3FF0000F4FF000002290000A6
:10415000B662FF1F8C62FF1F2863FF1F70B5160039
:1041600004AA148805AA15784A68507811780002C4
:104170002A4A0843801805284BD807F039FB031357
:104180001E29343F0720032C0BD80422121BAA42FD
:1041900000D92A0022491A803000091907F018FBBB
:1041A000002070BD0720112CFBD81222121BAA423E
:1041B00000D92A001B491A80EEE707200E2CF0D800
:1041C0000F22121BAA4200D92A0017491A80E3E7DE
:1041D0000720032CE5D80422121BAA4200D92A008A
:1041E00012491A80D8E70720032CDAD80422121BC0
:1041F000AA4200D92A000E491A80CDE70720032CD5
:10420000CFD80422121BAA4200D92A0009491A80D9
:10421000C2E700220A201A80C3E7C046DCD5FFFFB0
:104220007BBB0011D462FF1F6BBB001166BB00118A
:1042300061BB00115CBB001110B50D21024A03489F
:1042400006F04AFB10BDC04650BB00117442FF1F70
:1042500037B5012000F0CAF8204D214BEA89287CAF
:104260009A422AD1042201A900F074F9040000F056
:1042700031F9002C30D16B4699882B68C9BA4B4371
:104280002989184A1B145B1853806B46D9886B68C0
:1042900049BA89B24B4369891B0C5B181248191C37
:1042A0001BB2834200DD011C0B0400D500211388E2
:1042B00091800133138020003EBD0223002101AA1A
:1042C00000F01AF96A46040002230121287C063214
:1042D00000F012F90443CAE70124ECE7E862FF1F8B
:1042E000830500000063FF1F0F27000037B5012082
:1042F00000F07CF81E4D07226946287C00F02AF960
:10430000041E31D16B461B787F2B2DD800F0E2F8CC
:104310006B46D878F02302041B031A406B469B8837
:1043200014495BBA9BB21A432B68000953432A898C
:104330001B0C9B184B806B465A789B7812031B0111
:104340001A436B68024353436A891B0C9B181AB2C9
:104350001B0402D58C8020003EBD074B9A4201DC35
:104360008A80F8E78B80F6E700F0B4F80124F2E7E2
:10437000E862FF1F0063FF1F0F27000010B50F4CFE
:10438000237C002B0CD0382B0BD1012000F02EF811
:10439000CC22AC21207C920100F028F900F09AF8A0
:1043A00010BD074BE2899A42FAD1012000F01EF8B5
:1043B0000021207C00F0FAF8F0E7C046E862FF1F19
:1043C0008305000010B5084B1A7C002A09D05B69F0
:1043D000002B06D09847041E01D0FEF711FE2000E6
:1043E00010BD0124F9E7C046E862FF1F70B5002147
:1043F0000600162005F054FF0121152005F050FF9E
:1044000007F0B6F90400092007F04AF900222B4B07
:104410002B4DDA6661321A6019685B3A9143002EBF
:1044200028D0023A0A431A60AC4209D10A22DA6162
:1044300007321A6200221A639A630132DA6370BD8E
:10444000204A944203D11E22DA610532F1E71E4A66
:10445000944203D13022DA610632EAE71B4A9442E1
:1044600003D14322DA610832E3E7194A9442E1D1E9
:104470006922F7E702220A431A604622AC4203D0BF
:10448000104A944204D194225A6106329A61D1E7CB
:104490000D4A944201D1E622F6E70C4A944204D137
:1044A0003422FF325A610D32F0E7094A9442C1D1F9
:1044B000E62252005A610A32E8E7C0460050004046
:1044C0000024F4000048E801006CDC020090D003F6
:1044D00000D8B80510B50024064B0920DC6607F0AB
:1044E000E7F82100162005F06FFE2100152005F0E9
:1044F0006BFE10BD00500040F8B51C000023134DAA
:104500000F00EB666860160007F01AF8012380229E
:10451000EB6623002F615200013B08D207F018F927
:1045200008200B4A1168002C03D12000F8BD2A6135
:10453000F2E72B6F034203D02B69013C3370013645
:1045400013685B1A012BEED90124EEE700500040FE
:104550006008FF1F002370B5124D1400EB66686001
:104560000E0006F0EDFF01238022EB6623005200CF
:10457000013B08D207F0ECF808200B4A1168002C28
:1045800003D1200070BD2A61F2E72B6F034203D0F4
:104590002B69013C3370013613685B1A012BEED98D
:1045A0000124EEE7005000406008FF1F002370B5B3
:1045B0000C4C0D00E366606006F0C2FF0123E36669
:1045C000256107F0C5F88020074A80001168636BF9
:1045D000034205D113685B1A012BF8D9012070BD85
:1045E0000020FCE7005000406008FF1F002370B56A
:1045F000134C0E00E3666060150006F0A1FF012376
:10460000E36626610F33626B1A42FCD02B0A2361EA
:104610001023626B1A42FCD0EDB2256107F098F8C6
:104620008020084A80001168636B034205D113683B
:104630005B1A012BF8D9012070BD0020FCE7C046B1
:10464000005000406008FF1F002370B5124D0C00A1
:10465000EB666860160006F073FF0123A619EB668F
:104660000F33B4420ED107F073F880200B4A80005C
:1046700011686B6B03420CD113685B1A012BF8D9DC
:10468000012070BD22782A616A6B1A42FCD0013485
:10469000E7E70020F5E7C046005000406008FF1F34
:1046A0000A4B0B4A19689068884202D980235B0440
:1046B000C918536891601B1A5B181168D80B5B040A
:1046C00040185B0C106053607047C04628F00040F3
:1046D0001863FF1F10B51B4B1A793F2A01D93F22DF
:1046E0001A711979184A194811701822184902804C
:1046F00018480A8002804A809A79174880240280EC
:104700000C208A80013242432401101CA24200D9AD
:10471000201C124AC88010805A79002A01D1013227
:104720005A711A7A012A01D802221A725A791B7A0E
:104730000B4853430A21584306F072FE094C20608F
:1047400010BDC0460C63FF1F480AFF1F5C43FF1FDC
:104750002845FF1F5A43FF1F0465FF1F5843FF1FD3
:10476000710200002C63FF1F10B507210020FEF727
:104770002FFE124C002807D10C222000104907F010
:1047800027F8FFF7A7FF10BD0C2220000D49FEF708
:10479000F3FD0C2804D00C222000094907F018F87A
:1047A000094C0C2220000949FEF7E6FD0C28E8D050
:1047B0000C220021200007F00BF9E2E70C63FF1F39
:1047C000BCBB0011FC0C0000E862FF1FF50C0000F0
:1047D000F0B504000E00150085B0002A00D1BBE042
:1047E0000878002120706170262800D184E00FD85D
:1047F000072805D806F0FCFF5A3535353588968FE1
:10480000232800D1BFE025285ED0FF23637098E005
:10481000712800D18DE01ED8562851D0602800D1D3
:104820009CE05528F1D1013A874D0C2A46D8002A40
:104830000AD0711C280006F0CBFFFFF74BFF0C22BB
:1048400028008249FEF7D2FC0C222900601C06F0E9
:10485000BFFF0D2030E0722800D174E0DC2800D1C9
:10486000A9E0DB2800D0C3E0042DCED9B27873785C
:1048700012021A43F37810271B04134332791206ED
:104880001A430192052D05D06F1F3A000198711D42
:1048900006F09EFF05223100200006F099FF3A0045
:1048A0000199601D06F094FF781D05E00C222000A0
:1048B000674906F08DFF0C2005B0F0BD0C22B8E76B
:1048C0000C226449604DB5E7013A634D0C2A11D8BA
:1048D000002A08D0711C280006F07AFF0C2228005C
:1048E0005E49FEF783FC13222900601C06F070FF6E
:1048F0001420E1E70C22EDE7574D1322280007F0C2
:1049000067F8FEF77DFBEEE705225549601C06F0CF
:104910005FFF0620D0E712225249601C06F058FFC4
:104920001320C9E708225049601C06F051FF0920F6
:10493000C2E77178F72900D967E74C4B188801F076
:10494000BBFC0220B8E700F097FB012D02D0727883
:10495000474B1A6006F07CFF0020ADE7013A454D59
:10496000062A0ED8002A05D0711C280006F030FF58
:1049700000F0BCFF06222900601C06F029FF07207A
:104980009AE70622F0E7013A3B4D042A11D8002AA3
:1049900006D02800711C06F0D3FE384B1B68AB60B4
:1049A000FFF77EFE04222900601C06F011FF05209F
:1049B00082E70422EDE7022A00D826E773786370C5
:1049C000B378A37077781B021F43032A05D0033DF9
:1049D0003900AAB2F01CFEF709FC10223900E01CD5
:1049E000FEF7CAFC03000330002B00DB64E70DE791
:1049F000DA2800D009E7042D00D806E7B3787278EA
:104A00001B021343F27812041A4333791B06134333
:104A1000082D16D9B279717912020A43F179090485
:104A20001143327A12060A4303921A601B68052268
:104A300031002000039306F0CBFE0422601D03A981
:104A400073E7FE226270F1E70C63FF1FFC0C0000AD
:104A5000C8BB0011BCBB0011E862FF1FF50C0000D1
:104A6000F462FF1FD462FF1F9C44FF1F5E43FF1FC1
:104A700034F00040F943FF1F1863FF1F28F0004087
:104A800070477047013870B5042809D806F0B0FEA9
:104A90000309250812001B4B0221187806F0E8FFD5
:104AA00070BD184B0821187806F0AAFD0022164B9D
:104AB0001A72F5E70024144B124D08211A68287861
:104AC0001C8106F0D5FE2100287806F0C9FE0120E1
:104AD00000F044FE00F00AFFE2E70A4B08211878D4
:104AE00006F08EFD0948FFF7C7F9094B094A9B7983
:104AF00000209380084A13808022034B52001A81C1
:104B0000E6E7C0462863FF1F2C63FF1F6743FF1FB4
:104B10000C63FF1F2845FF1F0465FF1F020010B52F
:104B2000094B0A32094C92B2DA815A829881188272
:104B3000207802F027FA0422054B012120781A7010
:104B400006F096FF10BDC0462644FF1F6665FF1F96
:104B50006565FF1F10B5012909D1054B1B78002B96
:104B600005D02622034B04485A72FFF7D7FF10BD29
:104B70003865FF1F2C63FF1FC409000010B5164CD9
:104B80000A210223E05E06F04BFC00B200F002FEB8
:104B90000423E05E642106F043FC012100B200F032
:104BA0006BFE237A0024132220009A426041C0B297
:104BB00000F0E2FD032000F0A7FD200000F0B8FDAA
:104BC000064B1878053843425841C0B200F0C6FD84
:104BD00000F08CFE10BDC0460063FF1F6565FF1F1F
:104BE0000300F0B50A4D8E18B14202D15200801870
:104BF000F0BD0C782F6824093C5D0F271C700C78E1
:104C000001313C402F683C5D5C700233ECE7C046EC
:104C10005443FF1F10B5114B1A781870002A0ED09C
:104C200000280BD10E4B1A78062A07D85423D340FC
:104C3000DB0703D50B4B187802F0A4F910BD002850
:104C4000FCD0074B1B78012B02D0033B022BF5D87D
:104C5000044B0121187806F00BFFEFE73865FF1FC2
:104C60006565FF1F6665FF1FF7B5614D614A6249C3
:104C70002870082005F0DAFB0121022005F0D4FAA3
:104C8000022005F0BDFB0121002005F0CDFA002037
:104C900005F0B6FB00F054FEFEF7B2F906F000FC9A
:104CA000032256495648FFF79BFF2D240300042298
:104CB0001C7054490130FFF793FF30230222047027
:104CC00043708370504C514B2000DA8706F020FC73
:104CD000022815D0062220004D49FEF74DFB06287C
:104CE0000ED00321200006F053FC8D23E3706E3BB1
:104CF000237106221933200045496371FEF776FAC5
:104D00000D23444F444C454E3B70013B0422300080
:104D100043492370033B6370019606F059FD2D2330
:104D2000012240494048A371FFF75AFF01223F4941
:104D3000FFF756FF01223449FFF752FF0020FFF72B
:104D400069FF3B4E3B4A01213B4B1278307802F021
:104D5000DBF8230000213A78307802F0D5F8012200
:104D60002178364B01391A700020019AC9B205F03A
:104D7000D1FC334B1A68552A30D100221A60314BCE
:104D80003C3231485A72FFF7C9FE2021287806F0DC
:104D900047FE0120404205F009FD0120404205F098
:104DA000A5FDFFF749FAFFF74BF800F08BFC012057
:104DB0004042FFF715F9012006F08AFDF72001F0C7
:104DC0005FFA0121287806F053FE287802F036FABF
:104DD0001E4806F07DFBFEF741FFF7BDFA210B4BA5
:104DE0001B4A49019981DA8119825A82CDE7C0466E
:104DF0002863FF1F814A0011554B00119C44FF1F7F
:104E0000D462FF1FF462FF1F6509FF1F2644FF1FC6
:104E1000ADAC00003465FF1F1565FF1F1765FF1F50
:104E20007BBB00116709FF1F1C65FF1F6609FF1F81
:104E30006665FF1F8643FF1F6743FF1F0665FF1F51
:104E400034F000402C63FF1FC40900003863FF1FCB
:104E50004A1F0000F8B50A0020230D001A4019422D
:104E60003AD0454B1B78002B23D0FFF719FC434C5D
:104E7000434E6368727AC31A934202D36060FEF7AE
:104E8000EDFE327A217A531EDBB2994214D1FFF73C
:104E900075FA637A002B09D0013BDBB26372002BF9
:104EA00004D1707964335843FFF738FE237A013315
:104EB000237220206840F8BD9142EAD30023237278
:104EC000FFF780FAFFF75AFE2E4F3800FEF7D4FFA7
:104ED000390006F06DFDDCE70BB2002B0ADA2A4B35
:104EE000187806F03DFC002801D006F049FD80202E
:104EF0000002DFE70224214206D0204B01201A7273
:104F0000FFF788FE2000D5E70B0715D5FFF7C8FB94
:104F10001A4A1B495368497AC31A8B4202D350601C
:104F2000FEF79CFEFFF74EFAFFF728FAFFF726FE82
:104F300000F0E2FB0820BDE71024214206D00E4B12
:104F40001B78002BDED1FEF78FFFDBE70124214227
:104F50000AD00E4800F068F806F0CAFC072000F0FE
:104F600019FC00F0C3FCCDE70424080020402142D6
:104F7000A1D0FFF751F8C5E73865FF1F2C63FF1F6D
:104F80000C63FF1F6743FF1F2863FF1F4C43FF1F76
:104F9000F0B51B4B1B4F1B883A8804001A4E1B4D63
:104FA00085B09A420DD832889A420AD3184B1A8893
:104FB0002B889A4205D1174A174B12881B889A42B0
:104FC0001BD0052001F0B2F93B8802AA1380338878
:104FD000019053802B88114D93800F4B02A91B88A1
:104FE000D3800F4B2A78188802F0CEFE0D4B082193
:104FF0002878019A1C7006F0D3FA05B0F0BDC046BF
:105000000265FF1F5C43FF1F5A43FF1F0465FF1F1C
:105010000065FF1FFE64FF1F5843FF1F6665FF1FEB
:105020005E43FF1FFC64FF1F13B50C4B1C78002C64
:1050300011D1002801D00A4B18600A4A0A4B117896
:105040000A4A10780A4A01920A4A0092002205F0A0
:1050500059FA200016BD1124FBE7C0466565FF1F05
:10506000F864FF1F6465FF1F5465FF1F6665FF1F1F
:105070004065FF1F4465FF1F10B5064B12201B78CB
:10508000052B06D1044B13221988044B187801F024
:1050900029FB10BD6565FF1F5E43FF1F6665FF1F8F
:1050A00010B500240122114B52421870104B1C7095
:1050B000104B1A8002F0C2F804220F4B21001A7024
:1050C0000E480C3206F084FC102221000C4806F039
:1050D0007FFC07220B4B1C600B4B1C700B4B1C7096
:1050E0000B4B1A700B4B1C7010BDC0466665FF1F42
:1050F0006565FF1F5E43FF1F6465FF1F5465FF1F4B
:105100004465FF1F4065FF1F1465FF1F1365FF1FE8
:105110006043FF1F1265FF1FF8B5174C0600257886
:1051200006A814240078052D23D1B41F134FA5B26F
:105130001824BD421DD88D1FADB2BD4219D8FA2525
:105140006D00AA4215D21D000D4F0A3DADB2BD4201
:105150000FD80C4C26800C4C21800C4900240A806E
:105160000B4A1380FFF714FF0A4B0421187806F04E
:1051700047FA2000F8BDC0466565FF1F790C0000A6
:10518000750C00005C43FF1F5A43FF1F0465FF1F9F
:105190005843FF1F6665FF1FF0B50BB20D0089B0C5
:1051A000002B00DB76E1A64E307806F0D9FA041E1B
:1051B00055D00378A22B00D127E1D02B1AD0912B08
:1051C0004AD143780E2B47D19E4B82889A4243D1D5
:1051D0009D4A83681278052A3ED1032018567F28FD
:1051E0003AD09A4B1B68002B36D05B68002B33D02B
:1051F000984731E0807807282ED806F0F9FA042D78
:105200001D444479ADDD6378002B11D10622E11CE9
:105210008F4806F0DDFA01218B4B19708D4B1A78FF
:10522000002A5BD08C4B307801F06EFE002855D000
:105230000722854B1A7051E061780029F8D1E37894
:10524000002B11D0854A864B1278307801F05CFE35
:1052500060706378002BEBD1200006F091FB80207A
:105260000002684009B0F0BD774B1B78022BF3D0E9
:105270000121307806F024F90028EAD101213078A4
:1052800006F0F6FBE5E76378002BD1D16E4F0328DB
:1052900007D13B78052B02D101333B701EE002237E
:1052A000FBE7704B1A88704B0293002A0BD01B78D7
:1052B000002B03D00121307806F072F93B78062BE1
:1052C00004D1013BE9E7029B1A70F7E7042B41D1B7
:1052D0000121029B3078197006F0CAFB5B4B1B68FA
:1052E000002BB9D01B68002BB6D0574A10787FE747
:1052F0006378554F002B27D10622211D5B4806F00D
:1053000067FA62895A4B5B491A80A2895A4B1A8004
:10531000E3890B800521397058490A80584A138067
:10532000228A584B1A80584B1B78012B09D11F2019
:1053300000F0FCFFFA22920042430421307806F08C
:105340002FF90022484B75E7312B00D070E700227F
:10535000454B1A700323A0E706220021434806F0BC
:1053600037FB0023454A04211380454A30781380D7
:10537000444A138006F044F90821307806F040F9D9
:10538000A379083B5A4253412F4A03331370314BE0
:105390001B78002B06D0344B30781A78002A06D0C0
:1053A00001F0F0FD0122324B52421A8096E70121B2
:1053B000197006F05DFBF5E70821307806F020F95A
:1053C0006378002B00D047E72C4B2E4F0293E388E5
:1053D000029A042113802A4B307803932389039A7D
:1053E000138063893B8006F06BF8002800D033E718
:1053F000264B1B68002B00D12EE7039902983A88B0
:10540000098800881B68984726E74379132B00D04A
:1054100022E70389012B0AD11D4B1B78022B06D1F1
:105420000821307806F0ECF8FFF726FE14E7052097
:1054300000F07CFF08210200307806F0B1F80BE79D
:105440006665FF1F051400006565FF1FF864FF1FF8
:105450003965FF1F8643FF1F6743FF1F3465FF1F2A
:105460001565FF1F3665FF1F3865FF1F0765FF1FA6
:105470005E43FF1F0E65FF1F1065FF1F0265FF1FC4
:105480000065FF1FFE64FF1F0665FF1FF464FF1F1A
:10549000FC64FF1F8020C001014200D0E1E6CB0781
:1054A00031D5324B1B78002B1DD0314E05AC3378F3
:1054B000052B1AD1023B23702E4B21001B7823723F
:1054C0002D4B1B7863722D4B187801F0C1FC00281E
:1054D00009D007202A4B30701B68002B03D01B68B3
:1054E000002B00D098470120BBE60E20254B06225A
:1054F0001B7825492370254B1B78637002ABC018BD
:1055000006F066F9D8E7022308001840194209D0CE
:10551000174B1B78052B03D11D4B188806F010FA8A
:1055200002209EE60424214203D0FFF731FD200033
:1055300097E6082308001840194200D192E6154B5F
:105540001C78012C03D0022C0DD0082089E6124BC8
:10555000124A134913481B8812880988008800944E
:10556000FFF7DAFDF1E7FFF787FDEEE73865FF1F8C
:105570006565FF1F6043FF1F1265FF1F6665FF1F04
:10558000F864FF1F1465FF1F6143FF1F1365FF1FB2
:105590005E43FF1FFC64FF1F5843FF1F0465FF1F8E
:1055A0005A43FF1F5C43FF1F10B502A804880B205D
:1055B000002C10D1496808784978090201430C4849
:1055C000814209D1022119800A4B59881170DB7878
:1055D00000205BB2537010BD074C0A20A142FAD1E3
:1055E00002211980034B998811705B79F0E7C0465E
:1055F0006E2A00000063FF1F6F2A0000F7B5150038
:1056000008AA16884A680F4F14785278120222436B
:105610000A24BA4214D10122DBB2019200962A0078
:1056200005F076FE041E0BD1074B1B68002B07D03C
:1056300068782A780002104342425041013098476E
:105640002000FEBD022900007865FF1F30B501254E
:1056500003790400BFB02B4227D01549408805F0DC
:10566000C3F928420DD06A46124B69465B8D138000
:1056700002235380104B5B8893806088002202F0E5
:1056800079FA0E49608805F0AFF9C0070DD56A4672
:105690000B4B69461B88138002235380064B9B8863
:1056A00093806088002202F065FA3FB030BDC046AA
:1056B0007065FF1F8843FF1F0063FF1F6865FF1FA2
:1056C000E243FF1F10B5074C0749200005F042F9DF
:1056D0002000064905F03EF90721054A054805F076
:1056E000FBF810BDFFFF00007065FF1F6865FF1F1E
:1056F00048BC00118843FF1F10B5024803F0BCF8F6
:1057000010BDC0464D56001170B55F2508260749EB
:105710008400CA788B7840012A40B3433440A843C0
:10572000234302438B70CA7070BDC046F943FF1F0C
:10573000010043B204205A0002409B000C30034099
:105740001A43152310B5044CE0789843143B0B40E2
:1057500018430243E27010BDF943FF1F10B5054B1B
:10576000082419790A00A243002801D022000A4324
:105770001A7110BDF943FF1F10B5054B4024D978AD
:105780000A00A243002801D022000A43DA7010BDAB
:10579000F943FF1F0821F8B5324D334BAE780400B2
:1057A0000E40AE70984204DD67232B70473B6B7050
:1057B000F8BD2E4B984203DAE0232B703A3BF6E714
:1057C00000232B706B7083B21A0029485F3292B2AB
:1057D000284F82422CD9002C03DA5B421CB20423EE
:1057E0002B70053420B20A2105F01AFE04B2FA2308
:1057F0009B009C4232DB08232A7813432B706421E0
:10580000200005F00DFE0A2100B206F0B1F809B241
:105810002A787B5C13432B700A21200005F000FEE0
:105820000A2100B206F0A4F809B27B5C6A780AE0AB
:105830006970002CDBDA5B421CB204232B70F3226C
:105840006B78092CE8DC13436B700A21200006F00A
:105850008FF809B27B5C1E43AE70A9E7632CCEDCE7
:10586000EDE7C046F943FF1F1B4E00001DFCFFFF84
:105870002A0800006FBC00110823F7B5194FCD00AE
:105880003E7904001E403E71EDB2632806DD5F33B1
:1058900033433B7120231D437D71F7BD0300093362
:1058A00005DA20235B4233433B71A623F3E70E4B1B
:1058B000019300280BDA0423444224B23B710A21ED
:1058C000200006F055F8019B09B25B5CE3E709286C
:1058D000F5DD0A2105F0A4FD019B00B21B5C1E430F
:1058E0003E71ECE7F943FF1F6FBC001170B5104B20
:1058F0001B78002B1AD00F4E0F4D062231002800C6
:1059000005F0AEFE002811D0062231000B4C280015
:1059100005F016FF0020FEF769FD072221003E205A
:10592000FEF792FE002801D0FEF7D4FD70BDC04600
:105930008365FF1FF943FF1F7D65FF1F7C65FF1F08
:10594000002010B5FEF752FD0D223E200549FEF75E
:105950007BFE0023984200D13E33034A1370FEF7CA
:10596000B9FD10BD62BC00118365FF1F0200F0B5D8
:1059700001270A480A4E51188B1A002B00DCF0BD93
:10598000082415784308684038404000805B013C9B
:1059900058406D08002CF5D10132EDE7FFFF000003
:1059A00080BC0011F0B500250F269D4200DBF0BD44
:1059B0004C5D070944403440A400A05801357840AC
:1059C000F3E70000F0B589B06A460D000B000F2721
:1059D000110010351C780133260024093E40167052
:1059E00054700232AB42F5D12023024AFFF7DAFFAE
:1059F00009B0F0BD84BC0011F0B54E780B7889B0C9
:105A000036020C00170001901E43012A61D9974B02
:105A10009E4200D877E001339E421CD1062A17D15E
:105A2000CA788B7812021A430B791B0413434A7904
:105A300012061A438E4B5A6100221A705A808D4A00
:105A40005A608D4A9A608D4ADA60002009B0F0BD34
:105A500088225205EEE78A4B9E423CD184498B78DE
:105A6000002B00D0F9E00C2A31D10F22A378934308
:105A7000E278120213432279120413436279120668
:105A800013434B60E279A07912020243207A0004AA
:105A90001043627A12060243CA60E27AA07A1202C6
:105AA000024378484A81834208D80423704914226B
:105AB00001980B7005F08CFE1420C7E71201D21874
:105AC00089235B059A42F0D801238B70BDE7022A37
:105AD000FAD00523EAE76C4A01239642E6D1FFF7A4
:105AE000CBFA052F0CD9E378A2781B021343227955
:105AF00012041A4363791B061343644A0393136029
:105B000005F0A6FEA1E75A4D2B78002B9DD1AB786E
:105B1000002B00D1A3E02B8901339BB20093B34249
:105B200000D094E0132AD4D9CF7C8B7C3F02122181
:105B300020001F43FFF71AFF874200D091E0002E9C
:105B40003ED1E378A2781B0213432279E96812045C
:105B50001A4363791B06134303930A228B4213D122
:105B6000FF23A370E370237163716B89002B0AD14B
:105B7000E37B227C1B0212041343A27B1343039397
:105B80001B0901336B8100226B89002B8DD0002A09
:105B900069D1686837013818000B6B6900030390FE
:105BA000984205D9686105F033FDEB780133EB705D
:105BB00068681022A11C381805F04AFF2E8144E7BE
:105BC0006F89009A7B1E9BB293423CD1E378A27806
:105BD0001B02134322792E4E12041A4363796C6818
:105BE0001B0613433100042204A8039305F0F0FDC3
:105BF000211D0C2205A805F0EBFD012004A940425F
:105C00001034FFF7DFFE013F012F17D1039A0B235A
:105C10002861824200D049E704223100686805F01B
:105C200017FF042203A9686805F0F2FEE968039AE9
:105C3000FF23914200D139E7F73B37E72100FFF717
:105C4000C1FE1034DFE70923B742A2D82EE7009B3C
:105C5000B34200D9F9E6072328E7022326E7032306
:105C600024E7062322E70A2320E7C046FFFE0000C0
:105C70000044FF1F00000111FFFF0000504859368B
:105C800001FF0000FFFF001102FF000034F00040A0
:105C90000C44FF1F10B5034C0B000122210000F043
:105CA0006BFA10BD555E00110B8870B506000D0033
:105CB0000224162B11D92B000322094900F05CFAAB
:105CC000041E0AD1074B2A881B88191C934200D94D
:105CD000111C300089B200F0EFFA200070BDC04600
:105CE000815E0011DE65FF1F10B54A780400013A9D
:105CF0000B000220012A07D80A78002A04D00522C6
:105D00002000024900F038FA10BDC046AF5E001115
:105D10000A7810B50B0004000220002A04D00722E4
:105D20002000024900F028FA10BDC0465B5F001158
:105D30000A7810B50B0004000220002A04D00922C2
:105D40002000024900F018FA10BDC046C15F0011E2
:105D500010B5034C0B000B22210000F00DFA10BD12
:105D6000F15F001110B5034C0B000D22210000F073
:105D700003FA10BD6360001110B5034C0B000F2235
:105D8000210000F0F9F910BDBD6000110A7810B5CE
:105D90000B0004000220002A04D011222000024936
:105DA00000F0EAF910BDC046CD600011002310B527
:105DB0001322190000F0E0F910BD000010B5034CEB
:105DC0000B001722210000F0D7F910BD1F61001150
:105DD000002310B51922190000F0CEF910BD000003
:105DE00010B5034C0B001B22210000F0C5F910BDBB
:105DF00059610011F7B584890D0006000121002CBE
:105E000022D000238268D3561778002B1EDA0C2C80
:105E10001AD90C3CA4B2131940880093230002F055
:105E200086FE431E984101307B06DB0F6B703F23DB
:105E3000013C1F40A4B22870AF70AC80002C07D08A
:105E4000B3680133AB6000210800FEBD0020EBE722
:105E5000AC60F8E70B7803704B8843704B881B0AE3
:105E600083700B79C370042070470420022B06D185
:105E70000020537811781B02009A0B43138070475F
:105E80000B8803700B881B0A4370022070470420A4
:105E9000009983420AD1537810781B0203430B8088
:105EA000D37890781B02034300204B807047F8B5ED
:105EB0000D004B7801240021461C03702B788B4287
:105EC00001D82000F8BD6B78B01C4F1C012B10D1FD
:105ED000890069184B88022233704B88B9001B0A6D
:105EE0007370691805F074FC04360434A4B2F9B276
:105EF000E4E7122359436B185A88043132705B88E7
:105F000010221B0A7370691805F062FC12361234F5
:105F1000ECE770B5049D14001E00052B01D8042089
:105F200070BD637812781B0213432B80E378A2784C
:105F30001B02134302226B802A71211D681D063E3D
:105F400005F046FCB2B22A81F02AE8D82800A11D4B
:105F50000A3005F03DFC0020E2E7002310B50A7886
:105F60009A4201D8900010BD9A008A1854880133D3
:105F700004705488DBB2240A447094888470928838
:105F8000120AC2700430EAE710B51100029C062B19
:105F900004D004201022142B01D010BD0222227143
:105FA0004B7808781B0203432380CB7888781B0248
:105FB000034363800431601D05F00AFC0020ECE718
:105FC00010B50C788B7804315C43E4B20370220086
:105FD000013005F0FDFB601C10BD0420022B06D132
:105FE0000020537811781B02009A0B4313807047EE
:105FF00010B50C000A88023105F0EAFB208810BDBC
:1060000070B504000D0004981100012B01D8042084
:1060100070BD167852781202324302800200F832C4
:1060200055701470E825002C00D10C35023B9AB253
:106030004280AA42EBD80231043005F0C9FB0020AF
:10604000E6E70420009983420AD1537810781B02B6
:1060500003430B80D37890781B02034300204B80CE
:10606000704710B50C000A88023105F0B1FB20889A
:1060700010BD000070B501211E000420049C0E40DC
:106080000B4218D1CB40DDB28D4214D90A49DBB2A4
:10609000098899420FD32300F6331D70330058004E
:1060A00011184978165C0902314301332152D9B2E3
:1060B0008D42F4D8002070BD2044FF1F10B50C00A5
:1060C0000A88023105F084FB208810BD10B50C78D9
:1060D0008B7804315C43E4B203702200013005F098
:1060E00077FB601C10BD10B511000298032B01D87E
:1060F000042010BD14785278043B1202224302801F
:10610000CA788C781202224342809AB28280F22AA4
:10611000EED80431063005F05BFB0020E9E710B54E
:106120000C000B8803700B881B0A43704B8883702C
:106130004B881B0AC3708A880430063105F048FB7F
:10614000A088043080B210BD0420012B03D10020B0
:106150001378009A1370704710B50C000B88037009
:106160000B881B0A43704A880230043105F030FB6B
:106170006088023080B210BDF0B589B003931E4B29
:10618000029242000700D05A019102F020F8132534
:10619000061E2DD0029B01240370019B002B04D00E
:1061A000001903999847001984B26B461B7A5BB2B9
:1061B000002B0FDA1021380002F01CFB19250028F3
:1061C00013D130003219E1B202F066FC051E0CD189
:1061D0000C34A4B2042304AA380005A993800696BF
:1061E000948101F0AFFD051E02D0300005F098FA51
:1061F000280009B0F0BDC046DC65FF1F70B5050082
:106200000C0000280CD00020814209D01022200070
:10621000044905F0DDFA01202B7823736B78637352
:1062200070BDC046C4BC0011F0B506000D001700DB
:106230001C0085B002291BD00020102907D1022B99
:1062400007D0102B03D115E00020102C08D005B08A
:10625000F0BD69463800FFF7D1FF2A0069460BE020
:1062600069463000FFF7CAFF22006946380004E0A3
:10627000022BE9D12A003900300005F009FBE6E7DE
:10628000031CF72800D9F723032008499AB2013AE2
:106290000B80D317034006499B189B100B80D30F2C
:1062A00004499B185B100B807047C0462444FF1FB5
:1062B0002244FF1F2044FF1F034B1B888B4202D345
:1062C000024B4000C15270472444FF1FDC65FF1F92
:1062D000014B4000185A7047DC65FF1F1722014B25
:1062E0001A807047DC65FF1F70B505000E2005F0B1
:1062F00067FA041E13D0D023037000230622837094
:1063000007494570033005F063FA064B2100DA8A2D
:1063100062811B7E2373044B187805F041FA70BD2F
:10632000F865FF1FE865FF1F7444FF1F262803D888
:10633000024B4000C05A70470148FCE72644FF1F4B
:10634000FFFF000070B506000C00094D1C22002163
:10635000280005F03DFB074B1E70074B1C7005F035
:106360006FFB0123002801D0002312202B7070BD89
:10637000E865FF1F7444FF1F0966FF1F70B5050025
:106380000D4C0800E260A16010220021656005F05C
:1063900077F9012803D11021A06802F058FD1022DE
:1063A0000021280005F06CF9012803D11021606854
:1063B00002F04DFD70BDC046E865FF1F70B5041EBC
:1063C00005D1002903D006220D4805F001FA0D4B36
:1063D0001D78012D11D1002C05D102221A7005F073
:1063E00027F8280070BD00221A70074B1B78FF2B7E
:1063F000F7D02000FFF778FFF3E70025F1E7C0466C
:10640000F865FF1FE865FF1F7444FF1F030010B508
:10641000002801D1002010BD00780B4A002803D1CC
:106420005988D1821B7913761378022BF2D100237D
:10643000984200D103331370044B1B78FF2B01D01B
:10644000FFF752FF0120E6E7E865FF1F7444FF1FD6
:10645000002911D000280CD04B79012803D140220B
:106460005242134303E03F221340032802D001208D
:106470004B7170474022F4E70800FAE770B5094D08
:106480000100287800280BD0074C0622200005F0D8
:106490009FF921002878FFF7DBFF200005F0B0FA14
:1064A00070BDC0460866FF1FE265FF1F00290AD0C5
:1064B000012808D13F224B799343C02B03D0403BA6
:1064C0005A425341981C704770B5174D06002B78FF
:1064D000FF2B15D00A2005F073F9041E10D0D0232D
:1064E0000370C83B8370114B11491B784670C37011
:1064F0000622043005F06CF92100287805F050F9E7
:106500000C4B1B78012B0DD10B4B1B68002B03D0C0
:106510009B68002B00D09847084B04211878084A44
:1065200005F0A6F970BDC0467444FF1F0866FF1F42
:10653000E265FF1F0466FF1F3066FF1F3466FF1F02
:1065400060EA0000014B98687047C046E865FF1F8D
:10655000014BDB6818687047E865FF1F074B10B5F3
:10656000DA68136801331360054B1878FF2803D0ED
:106570008021C90105F07CFA10BDC046E865FF1F07
:106580007444FF1FF7B50E0002F0C8F8051E1CD0BA
:106590000E4B06621F78002F00D10778AB791020D0
:1065A000019305F00DF9041E0FD0D0230380C73BE3
:1065B0008370019BE91DC3700622043005F008F9C1
:1065C00021003800E66005F0EBF8F7BD7244FF1FCC
:1065D000014B18787047C0460866FF1F054B00281E
:1065E00005D1054B1A78054B002A00D1014B180044
:1065F0007047C046F865FF1F0866FF1FE265FF1F72
:10660000014B58687047C046E865FF1F024B186889
:10661000431E9841C0B270470C66FF1F421E030024
:106620000120152A03D9FF3B5A425341D8B2704783
:10663000F0B51C0000230E0085B0039002920B7091
:10664000029A934201D3002019E0E55C5A1CD2B2B1
:10665000002DF8D0029851198142F4DC0233DFB2E8
:10666000A35C18000193FFF7D9FF002807D0013D74
:10667000019A0399EBB233708A4202D1E01905B056
:10668000F0BDDB19DBB2DBE710B50C0002F09EF8C1
:1066900003001220002B03D02100588805F0F0F8E9
:1066A00010BD000070B50E4D84006359002B15D04D
:1066B000186A002801D005F0A3F82B59586A002861
:1066C00001D005F09DF82B59986A002801D005F0FB
:1066D00097F8285905F094F800232B5170BDC04657
:1066E0001866FF1F1C4B70B504000E001500994280
:1066F0000AD11A4B1B68002B01D1122070BD1B68F8
:10670000002BFAD09847F9E7154B994215D1134B56
:106710001B68002B0AD01B68002B07D09847002865
:1067200004D1104B1C70104B1D70E7E729002000AE
:10673000FFF7AAFF0028E1D1F3E7080001F0EEFF20
:106740000028DAD003780320A342D7D129003000F3
:1067500005F096F8D2E7C046FEFF00001466FF1F62
:10676000FFFF00001166FF1F1066FF1FF7B5040052
:10677000808801F0D3FF0025A84203D00578A088C7
:1067800002F008F81C4E3378002B1FD0AB421DD10D
:106790001A4B28001978FFF777FF002818D000233C
:1067A0003370A3790820A778A688019305F008F82C
:1067B000011E0DD0D0230370CA3B8370019B47702C
:1067C00086808371280004F0EBFF01E0002DE8D102
:1067D000A0880B4B8200D358002B01D0FFF762FF3B
:1067E0001721A088FFF768FDA08801F027FDA08889
:1067F00001F0FEFDF7BDC0461166FF1F1066FF1FCA
:106800001866FF1FF0B587B01D000CAB1B88070092
:1068100001930DAB1B88142002930EAB1B8816004E
:1068200003930FAB1B880091049310AB1B88059357
:1068300004F0C6FF041E1AD0D0230370CB3B477070
:106840008370C670062229000430002D11D004F098
:10685000BFFF019B21006381029B0098A381039BE2
:10686000E381049B2382059BA37404F099FF07B086
:10687000F0BD05F0ADF8ECE7F7B5009308AB1B8869
:1068800007000C200D001600019304F099FF041E70
:1068900013D0280001F042FF00280FD00078D02349
:1068A0002370C93BA370009B21002381019B67706B
:1068B000A580E680638104F073FFF7BD014B187873
:1068C000EDE7C0467444FF1F13B5040064890389D3
:1068D000C2888188C0780094FFF7CEFF13BD000006
:1068E00010B5044C2068002803D004F089FF002371
:1068F000236010BD1C66FF1FA122F0B581889200A5
:106900004A43384B384F1B6804009B189D22920065
:106910009B18827989B01A603B68002B5FD01D7884
:10692000324B1B68002B04D05B68002B01D0002089
:106930009847260008363100E079FFF7B7FD237D40
:10694000E0710200E0780493638A29000393238AAC
:106950000293E3890193A38800933300FFF752FF6A
:10696000E378002B0BD1E289A379A18802920196EA
:10697000E27928000092012201F0DAFEE0703B6823
:10698000002B20D0FFF7ACFF194D287800281AD033
:10699000184B1978FFF778FE002814D02B78E6788A
:1069A00008200793A78804F00BFF011E09D0D0230D
:1069B0000370CA3B4670837087808671079804F025
:1069C000EFFE00232B701721A088FFF775FCA0882D
:1069D00001F034FCA08801F00BFD09B0F0BD064BBE
:1069E0009DE7C0463409FF1F1C66FF1F3066FF1F6E
:1069F0001166FF1F1066FF1F7444FF1FF8B50700E4
:106A000008000E0001F08AFE041E18D02620FFF7B1
:106A10008DFC051E00D12578062004F0D1FE041E51
:106A20000DD00021062204F0D3FFD0232370C23BF7
:106A300021006770A370A680E8B204F0B1FEF8BD33
:106A4000F0B585B001930AAB1B78070002930BAB3E
:106A50001B7808000D000092039301F05FFE061EF4
:106A600022D0102004F0ACFE041E1DD01022002104
:106A700004F0AEFF2620FFF759FC002800D1307843
:106A8000D0232370C13BA370009B21002372019B84
:106A900067706372029BA580A372039BC0B2E3720E
:106AA0000C9BE36004F07CFE05B0F0BDF7B50D0073
:106AB000019001F033FE071E20D00E2004F080FE6E
:106AC000041E1BD02620FFF731FC061E00D13E78A5
:106AD000D0232380C53B0622A370F91DE01C04F0DF
:106AE00077FE019B2A0063810123DD401A401D408F
:106AF000210022736573F0B204F052FEF7BD00006E
:106B0000F0B585B0029010000D0017000A9E0393A7
:106B100001F004FE041E31D0029B002B2ED1039BFA
:106B200002795B0724D5122313430422002E08D1D7
:106B30000B99002905D10C99002902D10D99002942
:106B40001AD01A430D9B2271002B00D0C9E0002EF1
:106B500000D1CFE0002D00D0CCE0606A002801D049
:106B600004F04EFE1C21300004F062FD606205E07E
:106B700002239A430E33D7E793432371654BBA0040
:106B8000D458002C00D1AAE0002E10D0236A002B8C
:106B900003D11C2004F014FF20625E4BBA00D358CE
:106BA000186A002803D01C22310004F011FE0C9B4F
:106BB000002B12D0574CBB001D596B6A002B03D120
:106BC000162004F0FDFE6862BB00E358586A0028F6
:106BD00003D016220C9904F0FBFD0D9B002B11D065
:106BE0004C4DBC006659B36A002B03D1142004F04D
:106BF000E7FEB0622B59986A002803D014220D9941
:106C000004F0E6FD380001F089FD051E67D0414B18
:106C1000BA00D358002B62D01A6A3420002A00D15F
:106C20001C389A6A002A01D0143080B20B9A002ACC
:106C300001D01C3080B25B6A002B01D0163080B2CC
:106C400004F0BEFD041E4AD01822002104F0C0FE4C
:106C50002620FFF76BFB0190002801D12B780193D0
:106C6000D0232370029B200063700A23294EA37057
:106C7000039BBD00A371AB59A780196A1830002986
:106C800005D01C22A06004F0A3FD2000343073590D
:106C9000996A002907D0030014221433E06002939C
:106CA00004F096FD02980B9B002B08D003001C22D9
:106CB0001C330B992061029304F08AFD02987359EA
:106CC000596A002903D01622606104F081FD6B46E9
:106CD0002100187904F064FD3800FFF7E3FC05B0EB
:106CE000F0BD10220D9B0D991B69A018236204F0C2
:106CF0006FFD2CE70B9B002B00D13FE7012D00D04F
:106D00003CE7606A002801D004F07AFD1C210B9852
:106D10002AE7C0461866FF1F10B5044C20680028FB
:106D200003D004F06DFD0023236010BD0C66FF1F2F
:106D30000B4B07B51A68002A01D100200EBD694629
:106D4000531C012012780731FFF772FC0028F4D0A1
:106D500002780123100018401A42EED0EEE7C04638
:106D60002866FF1FF0B51F4F01203B6887B0002B3E
:106D700025D09B78059300F0B3FB002821D00A2092
:106D8000FFF7D4FA04000B20FFF7D0FA164B0500EA
:106D90001E78731E9E413B68F6B2191DD878FFF726
:106DA00057FB3B682900DA7A043303929A790193FE
:106DB0000292009033002000059A04F0D1FD07B044
:106DC000F0BDFFF7B5FF002805D00620FFF7AEFAAB
:106DD00004000720D8E70820FFF7A8FA04000920DC
:106DE000D2E7C0460C66FF1F0866FF1F70B50A4E4B
:106DF000040033780D00FF2B0DD0042004F0E0FCDC
:106E0000011E08D0D0230370CE3B45708370C47040
:106E1000307804F0C5FC70BD8444FF1F70B50400D9
:106E200006200D0004F0CCFC011E0AD0D023037014
:106E3000CD3B8370054B44701B688580187804F047
:106E4000AFFC002C01D0FFF767FF70BD0C66FF1F81
:106E5000F8B5264F06003B680D001124002B05D124
:106E60000522234B1B78134202D112242000F8BDC7
:106E7000204A10241268002AF8D01278002AF5D08F
:106E8000DB0719D52B789A1E012A1AD80C2004F09A
:106E900097FD132438600028E8D000230A224370AD
:106EA00029000670023004F093FCFFF75BFF041E1C
:106EB0000AD0FFF731FFD9E700F012FB0028E1D13B
:106EC000E4E7002BE2D0D0E70B4B1B78032BCDD1AE
:106ED0001D20FFF72BFA094B18800028C6D0084B5D
:106EE00004211878074A04F0C3FCBFE70C66FF1FB3
:106EF0000966FF1F2866FF1F0866FF1F0666FF1F43
:106F00003466FF1F60EA0000F7B50193194B1400C7
:106F10001A78052306000F0012201A4221D00129F9
:106F200020D1154B1D68002D1BD002201F2C18D816
:106F3000002C02D0019B002B13D0104B1F221E707F
:106F40006E1C0021300004F043FD01992200300046
:106F500004F03EFC310020002C70002F06D004F01D
:106F60003FFCFEBD064B12201D68DCE704F038FB39
:106F7000F7E7C0460966FF1F2866FF1F8444FF1F0E
:106F80002466FF1FF8B50F4E12243368002B17D06C
:106F90001B780F3C834213D100250B4F0221387818
:106FA00004F02EFB094B042138781D8004F028FBE7
:106FB000074B28001D8033685C7004F099FA0400C8
:106FC0002000F8BD0C66FF1F3466FF1F2066FF1F00
:106FD0000666FF1F70B5012823D11B4C2388002BA8
:106FE00003D01A4A1578002D07D0194B1B68002BC7
:106FF00002D01878FFF7C6FF70BD3B2B02D93C3B8F
:107000002380F9E7134E0221307804F0F9FAFA22CE
:107010002388920002215A43307804F0C1FA258077
:10702000EAE70B4B1B68002BE6D00B4B1B785B078A
:10703000E2D5084B0221187804F0E2FA0022024B54
:107040001A80FFF769FED7E72066FF1F0466FF1F5F
:107050000C66FF1F3466FF1F0966FF1FF8B51E4D43
:107060002868002803D004F0CBFB00232B601B4EC4
:107070003068002803D004F0C3FB00233360184FAE
:1070800005243B7818002040234221D0154800F009
:107090002BFA3B78234213D0202004F091FC286087
:1070A000002813D02022002104F092FC202004F0BC
:1070B00087FC041E306005D02022002104F088FCEB
:1070C000002004E0286804F09BFB2C601320F8BD2E
:1070D00000F00AFAF4E7C0462866FF1F2466FF1F87
:1070E0000966FF1F7844FF1F10B50A4C23681A1E5B
:1070F0000ED0002808D10130587004F0F9F90028AA
:1071000005D02368002B02D00021FFF787FE012263
:10711000100010BD0C66FF1FF7B5274E0500336841
:107120000191181E21D05C78244F012C30D1FFF73B
:10713000FFFD002825D02000FFF7F8F804004128C3
:1071400014D91F4B022118781E4A04F091FB1E4BE4
:107150003C3C1C80022233685A703B78002B14D1CF
:1071600028000199FFF75AFE0120FEBDFA22920085
:107170004243002AEED0124B0221187804F010FA94
:10718000E8E7FFF7D3F80200F3E700233B70EBE7F3
:107190003B78002BE8D1032004F012FB011E08D03D
:1071A000D0230370CC3B457083703368187804F0AB
:1071B000F7FAFFF7B1FDD7E70C66FF1F0466FF1F64
:1071C0003466FF1F60EA00002066FF1F10B51749F4
:1071D000838802008B4220D011D815498B4217D0EA
:1071E000144900205B1899B2012907D892681178D8
:1071F0005A425341D8B2FFF7F9FD012010BD0E4AA3
:1072000000209B1807229BB29A424041C0B2F5E78A
:1072100083681878FFF768FFF0E7836899785A78F1
:10722000090218781143FFF777FFE7E70A2000000B
:1072300006200000F8DFFFFFAFDFFFFF014B1870F3
:107240007047C0468544FF1F10B5064C207001F002
:1072500041FA207804F0ECFB0521207800F062FD73
:1072600010BDC0463466FF1F0BB273B50D00002B76
:1072700000DBC4E0884B187804F072FA041E0ED0CC
:107280000378912B0FD0A22B00D1A1E0834B18786B
:10729000FF2852D0210004F083FA00284DD180202D
:1072A0000002684076BD43780F2B76D013D8052BAB
:1072B00070D00E2BEAD18088794B98422BD8794B2D
:1072C00098421BD8784B9842E0D1A3681878591C93
:1072D000FFF774F838E03E2BD8D18378032B74D0B5
:1072E0006CD8012B6ED0022BD0D1704B1B68002BB9
:1072F00023D05B68002B20D098471EE06C4BC01851
:107300000C28C3D804F04CFB1DC2C2150BC20B0BDA
:107310000B3223C23C00674BC0180728B6D8664B17
:107320001B68002B09D01B68002B06D02000984753
:107330000AE0A3681878FFF7C7F8200004F020FBE4
:10734000ADE7A068FFF762F800289FD0F5E7A368D3
:107350001B78002BF1D0554B1B68002BEDD01B6820
:10736000002BEAD0210055489847EDE74F4B1B68AA
:10737000002BE2D01B68002BDFD021005048F3E740
:10738000504B1B68002BD8D05B68002BD5D0210058
:107390004348E9E7FFF7EAF9CFE780884A4B98428C
:1073A00003D04A4B984200D070E7464B1B68002B35
:1073B000C3D05B68002BC0D02100D5E7153B012B63
:1073C000BBD963E7FFF798FAB7E7FFF77DFAB4E7B1
:1073D0003F4B1B78042B07D100236A4613800179A9
:1073E000408800F0C5FCA8E7364B1B68002BA4D0F2
:1073F0005B68002BA1D00100364898479DE7012427
:1074000021420AD0294B1B68002B04D05B68002B5B
:1074100001D000209847012043E78B070AD5264B6F
:107420001B68002B04D05B68002B01D0200098471C
:10743000022036E70421280008400D4200D131E740
:10744000254E3388002B21D0013B9BB23380002B8B
:107450001AD1FFF7DBF800280AD0204B1C70164B1E
:107460001B68002B04D05B68002B01D020009847DC
:10747000FFF7C6F8694601F001FD6846FEF7FEFF1A
:107480001D20FEF753FF308004200AE7024B1878D6
:1074900004F0B6F8F8E7C0463466FF1F8544FF1FC6
:1074A0000E20000001200000091000002C66FF1FC4
:1074B000FEDFFFFFAFDFFFFF3066FF1F0C20000085
:1074C0000B2000001466FF1F0D2000001320000099
:1074D0000966FF1FFFFF00000666FF1F0466FF1F0F
:1074E00010B501F09BF910BD014B18607047C04604
:1074F0003066FF1F0B880020162B01D817230420AD
:10750000014A13807047C046DE65FF1F00207047A8
:10751000074A03001188814207D0918800209942D0
:1075200002D101308000101870470020FAE7C046F1
:107530003C66FF1FF0B58F7806000D00C7B01E2F08
:1075400015D1FFF7E5FF051E03D10024200047B049
:10755000F0BD00223B003100C078009200F0B2FB89
:107560000400A81C00F0D3FBFF23EB70EEE7264BD2
:10757000062403931B78FF2BE8D0182FE6D87B084E
:10758000224A013BDB0002929A589446002ADDD041
:10759000029AD3185B68002BD8D00878002802D153
:1075A0004B78012B02D10624122FCFD107AFAB8825
:1075B000697800976446AA68A047041EC6D1AB78D4
:1075C000029A5B08013BDB00D318390030005B688E
:1075D0009847041E0BD1AB78042BB6D0039A310028
:1075E00010782200009700F06DFB0400AEE76A7887
:1075F000002AABD1AA7805A93B88087130000A702F
:107600004B80FEF747FBA0E78844FF1FD4BC001166
:107610001D4B37B5050098420BD000290AD1FFF762
:1076200077FF002805D11948FFF772FF002800D026
:10763000058037BD01291AD1FFF76AFF041EF8D073
:1076400001235B420380A378FF2BF2D0FE2B07D0EF
:107650000023E0781422009329001E3300F032FB4F
:10766000A01C00F054FB01235B426380E1E7022988
:10767000DFD1013901F0BEF80028DAD12800FFF788
:1076800047FF041EDFD1D4E7FEFF0000FFFF00002C
:10769000022210B5074B52421A80074801325A8025
:1076A0009A80DA8000F07EFA044801F025F8002084
:1076B00010BDC0463C66FF1F3575001111760011E4
:1076C0000388F7B50400002B02D102252800FEBD77
:1076D00042680221137825485268FEF7A5FD00286C
:1076E0002ED0234F01253A88002AEFD0802321880D
:1076F0005B0201259B1A9942E8DC0C2004F060F93A
:10770000061E31D03B8822889C4600231800019534
:1077100061469DB2491989B2AA421BD8002801D0FE
:1077200062443A8000233000082208C0210004F09F
:107730004FF8104A1368002B13D100251660C5E7D7
:107740006268022113780C485268FEF76DFD00282C
:10775000C7D1BAE760681D01401941810133019822
:10776000D6E71A001B68E6E71325AFE742BD001114
:107770008644FF1F3866FF1F40BD0011014B187083
:107780007047C0468844FF1F14230A0010B51A40F2
:10779000194204D00122102101F048F810BD4B0617
:1077A000F9D4012088434000F8E710B514008B0697
:1077B00004D50122102101F039F810BD08230A0078
:1077C0001A40194202D14BB2002B0FDA102101F0FE
:1077D0002DF8002808D02300F9331B78002BECD0BB
:1077E000F8342378012BE8D10020E6E7032089074D
:1077F000FAD4E2E7F0B51F00184B85B01C68019081
:1078000002910392002C27D1200005B0F0BDA5689D
:107810003301ED186B89019A934211D3029A934276
:107820000ED8002F04D10A9B002B10D12C00EBE7BF
:107830003B002978039A6868FEF7F6FC0028F2D12D
:107840000136B6B2A388B342E1D82468DAE7A36868
:107850000A9A5B891380E9E70026F3E73866FF1F81
:1078600037B50C000A8849880123914217D3002AB2
:1078700015D0651D23792A0002210A48FEF7D4FCA1
:10788000102300280BD023796188208800242A0047
:107890000094FFF7AFFF0A23A04200D02300180096
:1078A0003EBDC04642BD001113B50A000888498894
:1078B000012388420BD8002809D00024137905320F
:1078C0000094FFF797FF0A23A04200D0230018007E
:1078D00016BD13B50A0008884988012388420BD8D1
:1078E000002809D00024137905320094FFF782FFA5
:1078F0000A23A04200D02300180016BDF0B58BB0BB
:1079000003904A8808880E000123824255D300283C
:1079100053D00023012704AC237000227188130088
:107920000092FFF767FF051E3ED02078002835D172
:107930002B78022B18D167706A8983000130E31815
:1079400080005A8069680222201803F041FF2378E2
:107950000133DBB22370042B19D93B006889013055
:1079600080B2002BD9D01FE002236370122358434A
:107970006A89231804305A8069681022201803F09D
:1079800027FF23780133DBB22370002BE5D10C4AAB
:107990006B899B185A425341DBB2DFE76378012BB6
:1079A000E4D12B78022BC7D022780A23002A04D0F6
:1079B00021000398FEF798F9002318000BB0F0BDE2
:1079C0000100FFFF0F4BF0B504001868002816D027
:1079D00083685D89A54207D88288AE18B44203DA6D
:1079E00012019A18934201D10068EFE71E005F89E7
:1079F0001036A74204D1002900D00D801800F0BD38
:107A00003300EFE73866FF1F70B505000C000888EB
:107A10000021FFF7D7FF03000120002B04D0220034
:107A20002800197AFFF7C1FE70BDF7B50C000025DC
:107A300001902300F6331B78AB4201D800200AE006
:107A40006B00E65A00213000E718FFF7BBFF002863
:107A500002D126800130FEBD017A0198FFF794FE25
:107A6000002802D03B882380F5E70135EDB2E0E73E
:107A700010B5040008880021FFF7A4FF03000120CF
:107A8000002B03D02000197AFFF77EFE10BD000006
:107A9000054B1B68002B01D1180004E09A6852893D
:107AA0008242F6D1988870473866FF1FF0B50E27DE
:107AB000002687B0039302ABFF183E8005001F4BE2
:107AC00040891400984207D02B78013000976A68EB
:107AD00080B2FFF78FFE060002212B7818486A68F3
:107AE000FEF7A2FB00280FD06C892000FFF7D0FF23
:107AF000002802D0013C0419A4B2039B002B00D043
:107B00001C80300007B0F0BD02212B780D486A6858
:107B1000FEF78AFB0028E7D102212B780A486A6821
:107B2000FEF782FB002807D0002EDED03B88A34260
:107B3000DBD17489013CDFE76C89DEE7FFFF0000E1
:107B400042BD001140BD00113EBD001110B50C003A
:107B5000FFF7DEFC03000220002B0AD0002C00D02F
:107B600023609B781720FE2B03D00138FF2B00D118
:107B7000002010BD73B50D0001A904001600FFF729
:107B8000E5FF172805D0002E04D129002000FEF7BC
:107B900027F976BD01221021200000F047FE0028C1
:107BA000F3D0F6E7014B18607047C0464866FF1FE8
:107BB00037B56B469D1D010004000222280003F02A
:107BC000BFFD2B88B02B0ED12379122B09D12300B6
:107BD000FF339B78012B06D10121608800F0E0F88B
:107BE00001E01B2BF8D037BD10B5054B04211870F0
:107BF00000F098F8FFF74CFDFEF770FB10BDC04693
:107C00004C66FF1F0020F0B50BB20F0087B0834217
:107C100034DA274B187803F0A3FD051E2BD0037828
:107C2000A02B25D103AE3100FEF7E4F8041E0BD1E2
:107C3000B378DB0724D51F4B06341B68002B03D019
:107C40003100688898470400A868002801D003F034
:107C500067FD002C08D1184A039B1340174A934232
:107C600006D0B3781B2B03D00121688800F098F868
:107C7000280003F085FE80200002784007B0F0BDA8
:107C80000F4B1B68002B10D0310068889847041EEA
:107C9000DAD07378002BD7D1B27801A90A704B8063
:107CA0000C716888FDF7F6FFCEE70624F1E7C046C1
:107CB0004C66FF1F4466FF1F00FFFF00000112001B
:107CC0004866FF1FF7B50190822040000D001700A5
:107CD0001E0003F075FD04001320002C12D0B02309
:107CE00020002370089BFC22677065802671083095
:107CF000002B08D0190003F06BFD2100019803F060
:107D00004FFD0020FEBD089903F062FEF5E710B5B7
:107D1000041E06D00078FD2803D803F0C1FEFF231F
:107D2000237010BD0A1F93B210B504000220032B6C
:107D300005D882400020024BD1529B189C7010BD88
:107D40006C66FF1F0B8870B5043B04000D00022019
:107D5000032B0BD80121200000F04CFD0300142060
:107D6000002B03D02900200000F0DEFB70BD0000D6
:107D700007B51300034A00920A00012100F02CFC11
:107D80000EBDC046AD7F001107B5019203220092DF
:107D9000024B0A00122100F049FC0EBD2B8000119D
:107DA00007B56B4601AA11800449D88008780633CC
:107DB000012802D1190003F033FC07BD4D66FF1FF7
:107DC0000C4B10B518700023FF210B4A1380138150
:107DD00093819380094A53801370517293819372F7
:107DE000D174D3821375517703F04AFE00F0FCF989
:107DF00010BDC0467C66FF1F6C66FF1F4E66FF1FEE
:107E0000F0B58DB06B46002003910C229B5E83423F
:107E100000DBB0E05D4B187803F0A2FC051E00D13A
:107E2000A4E00378902B00D09DE006AF01004688C7
:107E3000380000F013FA79680400002900D19CE0B2
:107E40003B88052B6ED13B89032B1CD905AC200048
:107E500000F0A2F86288172A61D83989131D994267
:107E600031D17968237804310291D90738D5607807
:107E700000F08EF9071E06D0002303712378012B32
:107E800008D0132B23D0A868002800D178E003F095
:107E900047FC75E06288029909A800F0A6F80290F4
:107EA000380000F08BF909AA2378387A0192002271
:107EB00031000092029A00F012F9380000F064F9E3
:107EC000029B002BDFD0300000F080F9DBE7037865
:107ED000032BD8D16288029909A800F0D6F8DEE712
:107EE000122B13D1029909A800F0B5F8021EEAD1AD
:107EF00027498B88002BC6D0887909A9237801915E
:107F000061780091310000F0EAF8BCE7002302AA92
:107F100093833000617809AAFFF72AFFB3E71D4B6E
:107F20000993F6E7042B02D09A1F012AABD8184A0E
:107F3000043B9B00995A0029A5D0D21890783100B3
:107F40003A0000F0AEF800289DD13B88042B03D006
:107F500001213000FFF724FF012C04D1A86800287C
:107F600001D003F0DDFB280003F00AFD8020039B15
:107F70000002434018000DB0F0BD012800D182E797
:107F800001213000FFF70CFFEDE7C0467C66FF1FC4
:107F90006C66FF1F010017000B7803704B7843706D
:107FA000CB788A781B021343438070470A8803000A
:107FB00002700A88120A42700A88012A06D14A8889
:107FC00082704A88120AC2700420704702208242DE
:107FD000FBD14A8804309A704A88120ADA708A887B
:107FE0001A718A88120A5A71EFE710B5040001204D
:107FF00082420CD94B780A781B02134323808342B8
:1080000006D1CB788A781B0213436380002010BD11
:10801000022BFBD1CB788A781B02134363804B7908
:108020000A791B021343A380F0E70B8803700B88C7
:108030001B0A43704B8883704B881B0AC3708B8864
:1080400003718B881B0A4371CB888371CB881B0A11
:10805000C3710820704703000120082A14D14A7810
:108060000878120202431A80CA7888781202024302
:108070005A804A790879120202439A80CA7988792B
:10808000120202430020DA80704710B5040001207C
:10809000022A05D100204B780A781B021343238063
:1080A00010BDF8B5060010200F00150003F088FB86
:1080B00004000120002C0ED0A0230C2229002380D4
:1080C0006780201D002D07D003F082FB21003000C7
:1080D00003F066FB0020F8BD03F07AFCF6E7F7B585
:1080E0001E00009008AB142017001D78019103F0CA
:1080F00067FB041E12D0A2230370019B47704380CC
:10810000099B057146710C220830002B07D019001D
:1081100003F05EFB2100009803F042FBF7BD0999D4
:1081200003F056FCF6E737B5041E0FD04388002B4A
:108130000CD00025C1881323007A172201950095E1
:10814000FFF7CDFFFF2365806372257037BD000008
:1081500010B50C4904004A88002A09D08B89002BED
:1081600005D00020CB8A0222834201D010BD01221B
:1081700013000A20434300204032C854C8184280EC
:108180000472F3E74E66FF1F0023438003707047BD
:10819000094B00211A0010B55C88002C06D01C7910
:1081A000844203D10A234B43D01810BD01310A3356
:1081B0000329F1D10020F8E74E66FF1F10B5040037
:1081C000407A03F06DFCFF23637210BD70470430EA
:1081D00010B580B203F0ECF9002803D00421494225
:1081E00003F03EFC10BD000070B50025104CA068E7
:1081F0002580A581A580A84202D003F091FAA56050
:1082000000250C4C0C4B606D1D80230058331D70F5
:10821000A84202D003F084FA656500256068002852
:1082200001D003F07DFA013508340A2DF6D170BD76
:108230001467FF1FB866FF1F0867FF1F70B5041E95
:1082400009D1054D2880A881A880A868002802D0FF
:1082500003F066FAAC6070BD1467FF1FF0B54B8881
:1082600085B00193002343600A7905000F00022ABC
:1082700000D07BE0CA88032A17D98B685E7819780A
:108280003602DC78D8790E4399781B7A24021B02D7
:108290000C43034353495BBA0B80331D93421ED1F9
:1082A000042C04D0631F022B0ED9012015E0019A83
:1082B0004D4B1201D35A002B06D00198FFF7BEFF99
:1082C0004A4A1369013313610421B8682E812C8056
:1082D000494203F0C5FB6860002005B0F0BD434D86
:1082E000042C06D0631F022B0FD9EB680133EB601F
:1082F000DBE7019A3C4B1201D35A002B05D00198C1
:10830000FFF79CFF2B6901332B61374B3000029341
:10831000019B029A1B010193002301998C468B5209
:10832000130063449C8003939E81FFF750FF039BDF
:10833000041E986016D00421B868494203F090FBEF
:10834000FA880100043A200003F042FA0199029AE7
:10835000FB888A5A043B9B18029A8B522B68013384
:108360002B60A2E7AB690133AB619EE71E4B029322
:10837000019B1E01029BF35A002B2DD002998C19F0
:10838000A068002828D0012A26D1FA889B189BB221
:108390007352A189994217D39B1AC018B96803F088
:1083A00017FA029BA289F35A934200D07DE700227C
:1083B0002B81A3882B80A3686B60029BF2520B4A2F
:1083C00053680133536070E7084A93680133936040
:1083D0000198FFF733FF68E7044A5369013353619B
:1083E000F6E7C0467E66FF1F1467FF1F8466FF1F07
:1083F00070B5051E15D10B4C0B4B1880230058335C
:108400001870606D002802D003F08AF965652500B8
:1084100050356068002801D003F082F90834AC427E
:10842000F7D170BDB866FF1F0867FF1FF0B51700D2
:10843000A12285B0920001934243394B06001B688C
:108440000C009B18D933FF331D78FDF741FF043032
:10845000854204DD3000FDF73BFF0430C5B2BD426C
:1084600007D33A0000213000019B03F029FA05B040
:10847000F0BD2900380003F06BFA2300C6B2503378
:108480001E700393019B29006365380003F010F808
:10849000CBB20293002B02D0039B01361E70002644
:1084A0002300503303931B78B34204D8606D002837
:1084B00031D10020DBE7029A2800002A04D0013BDA
:1084C0001000B34200D02800F700E719387003F01D
:1084D0000FF9786000280ED03A78019903F078F906
:1084E000019A3B780136D3180E4A0193D369F6B24C
:1084F0000133D361D4E7039B18706065A74205D1AF
:10850000084A1320D36A0133D362B0E7606803F0EE
:1085100007F90834F2E703F003F900236365C8E7BD
:108520003409FF1F8466FF1FF7B50D000700042103
:10853000686803F095FA2B89040003702B891B0AE5
:1085400043702B8883702B881B0AC3702E890225E9
:108550000436F6B2FB2E15D81B4B9F4214D10C20CB
:1085600003F02EF91135011E0CD0902303708E3BC1
:108570000371043B4380154B8460C680187803F078
:108580000FF900252800FEBD5C237B43104AD31859
:108590000093583301931B78002B0FD10300320056
:1085A00038000099FFF742FF019B05001B78002B64
:1085B000E8D13800009903F043F8E3E7054A0725BE
:1085C000536A01335362DDE7FEFF00007C66FF1F44
:1085D000B866FF1F8466FF1FF0B587B000901720B4
:1085E0000F0016000193FFF7F2FD1325041E19D0AA
:1085F0000C98031E02D00199201D9847030AE370CE
:10860000052302AAA070043090812770009866703C
:1086100003A993800494FFF787FF051E02D0200072
:1086200003F07EF8280007B0F0BD0000F0B587B079
:108630001F000CAB1B780391059301210DAB0600C5
:108640001C78049200F0D6F81425002821D02000D0
:10865000FFF77EFD0135041E1BD01149059B0A78EA
:1086600003700132D2B2131EC68001D101231A0059
:108670000B7022713000049B03990097FFF7ACFF49
:10868000051E09D1230021000648074A093303F0DB
:1086900027F9280007B0F0BD002363802370F8E7B6
:1086A0008066FF1F2781001130750000F8B50500B6
:1086B0000E00064C064F2368002B02D03100280024
:1086C00098470434BC42F6D1F8BDC0462467FF1F6A
:1086D0003867FF1F0123064A5B4253800023137152
:1086E0005362044A136053609360D3601361704710
:1086F0003867FF1F2467FF1F0200002310B50649DB
:108700009C000859002801D1625010BD0133052B8F
:10871000F6D11320F9E7C0462467FF1F034A5388A8
:10872000181A434258414042104070473867FF1FB3
:10873000F0B585B002930AAB1F780CAB1B88009094
:1087400008000E0001920393FFF7E8FF05001120D7
:10875000002D1BD10E48FFF7E1FF04001520002C6F
:1087600014D006220B99A771E01D03F031F8019B8C
:1087700030002371029B29006371009B6680237087
:10878000039B6562E381FFF791FF280005B0F0BD10
:10879000FFFF000010B5FFF7C1FF04000220002C0E
:1087A00012D060880121FFF781FF606A002801D0A4
:1087B00003F026F828220021200003F009F9012304
:1087C00000205B426380207110BD000030B5074A75
:1087D000074C5588010013780020A54204D05B1A8D
:1087E00059424B415842104030BDC0463867FF1FC8
:1087F000FFFF0000084A10B501230C00904208D08A
:10880000FFF78CFF031E04D0037923405A1E9341C7
:10881000DBB2180010BDC046FEFF0000024B187905
:10882000431E9841C0B270473867FF1F70B50400FF
:108830000D001600FFF772FF002804D10D4B9C427B
:1088400000D0143070BD416A03790520002907D09B
:1088500012221A40102A02D10520002EF2D10F2038
:10886000DB06EFD5897E0C20A94289414942494265
:108870000840E7E7FEFF0000030010B5002800D124
:1088800010BD0348034A41889142F9D09847F7E761
:108890003867FF1FFFFF0000002330B5C45CCD5CCC
:1088A0006C40D4540133102BF8D130BD0F2300227B
:1088B00010B5C45C64002243CA54C25CD209013BB7
:1088C000F7D210BD0200010010B52032103102F0C5
:1088D000A7FF10BDF0B58BB00390102005931700D3
:1088E000049103F06DF80090102003F069F8009BEC
:1088F00013240190002B05D000280CD113240098DC
:1089000002F07EFF019B002B02D0180002F078FFDE
:1089100020000BB0F0BD102003F052F8060010202C
:1089200003F04EF813240500002E00D1AEE000281D
:1089300019D01022002103F04BF8320029000398CF
:1089400002F06EFF041E0ED133787F2B51D8300019
:108950000099FFF7ABFF009B1B787F2B53D8019941
:108960000098FFF7A3FF300002F04AFF002D02D06D
:10897000280002F045FF002CC1D1102003F020F8A0
:108980000600102003F01CF80290002E7CD0002876
:1089900078D03A000F3223000125121105D00F3391
:1089A0003B4015B25A4253411BB26A1E1201002BC2
:1089B00033D0049BD2B298180099029AFFF76CFF4B
:1089C000013D10220021300003F002F8ADB2049FF7
:1089D0002D017D19AF4242D0002C33D0300002F07F
:1089E0000FFF029B002B00D189E7180002F008FF5F
:1089F00085E729003000FFF759FF28002549009A34
:108A0000FFF74AFFA7E729000098FFF74FFF28006C
:108A10002049019AFFF740FFA5E70F210F40049975
:108A20008A18D9B28F4208D9D15C06A819540133EB
:108A3000102BF6D1029A0199C0E7791A48424141B8
:108A4000C901F2E73900300006AAFFF725FF32001E
:108A5000039806A902F0E4FE10370400BAE7002CE0
:108A6000BCD13000029906AAFFF716FF320006A912
:108A7000039802F0D5FE082204003100059802F0A8
:108A8000A7FEABE71324A9E71324AAE7002800D028
:108A90006EE733E748BD0011F0B58BB00F0016004C
:108AA0000225009000283FD0002A3DD00B1DDBB2EC
:108AB0001800029302F084FF1135041E34D0FDF734
:108AC00047FD05003A000099201D02F041FDEBB280
:108AD0000393E3702B0CDBB22F0A00936370FFB299
:108AE0002B0E2370A7700193FDF72CFD10220100BF
:108AF00006A802F02DFD2100029A04AB06A8FFF79C
:108B0000E9FE051E0DD1039B08223370009B04A9CA
:108B1000B370019B7770F370301D02F019FDFDF703
:108B20001DFD200002F06CFE28000BB0F0BDF0B57A
:108B30008FB00D00149E039004920593002A03D178
:108B4000022420000FB0F0BD002EF9D00398FFF7EB
:108B5000E5FD1424071EF4D07278337812021A430C
:108B6000B3781B041343F27812061A43036A019286
:108B7000934201D30133E3D1002D03D03B7901248B
:108B80009B07DED50822002106A802F021FF059BE5
:108B900013240433DBB21800029302F011FF051E08
:108BA000CFD0059A0499043002F0D2FC042231009F
:108BB000280002F0CDFC3900102210310AA802F082
:108BC000C7FC2900029A06AB0AA8FFF783FE041E21
:108BD0000FD1082206A908A802F0BAFC0822311D0C
:108BE00008A802F055FE012807D101990398FDF766
:108BF000C9FC280002F004FEA3E70124F9E7000005
:108C000070B51C4C05002368181E10D0002D14D11F
:108C10001A78002A0CD1981C083202F0D9FD02F013
:108C200017FD0135002808D123681D70012070BD93
:108C30000A331800082202F0CBFD2368002BF5D080
:108C4000122002F0BDFD061E0DD0C1232168037065
:108C5000457002311022023002F0BAFD2368310063
:108C6000587802F09DFD206802F0CAFD00232360C1
:108C7000DCE7C0466067FF1FF8B504002020FDF761
:108C800055FB0D4EA700BB590500002B0DD0002849
:108C90000BD0D878FF2809D108492A000C55F35980
:108CA00007480333611802F01BFEF8BD290002F0EB
:108CB000C7FB0028F0D1F8E77C67FF1F6467FF1F40
:108CC000D19E001170B5064D84006359002B05D06C
:108CD000D87802F0E5FEFF226359DA7070BDC04615
:108CE0007C67FF1F70B506008CB00C0015000021DA
:108CF0003022684602F06CFE31001022684602F015
:108D000027FC1D2021000322684402F021FC684654
:108D1000FFF7D8FD2D21040003222800694402F04A
:108D200017FC20000CB070BDF0B50700160097B01E
:108D300001931CAB1D7830221EAB00910AA80021C4
:108D40001C7802F045FE102239000AA802F000FC4F
:108D50001022002102A802F03BFE0722310002A8E7
:108D600002F0F6FB072202AB9818631E9C410199A2
:108D700002F0EEFB02AB9C732B005A1E934102AA39
:108D8000D3730021102206A802F022FE06221D99AC
:108D900007A802F0DDFB1A2002ABC01806221F99BB
:108DA00002F0D6FB102200990EA802F0D1FB10228F
:108DB00002AB0EA908781C78013A6040D2B2087064
:108DC00001330131002AF5D10AA8FFF77BFD1022FB
:108DD00012A904000EA802F0FBFC102206AB0EA99B
:108DE00008781D78013A6840D2B208700133013129
:108DF000002AF5D10AA8FFF765FD04431022209848
:108E0000E4B212A902F0A4FB200017B0F0BD70B5C7
:108E10000E0014008CB00100102268461D0002F004
:108E200097FB3100082204A802F092FB21000822DF
:108E300006A802F08DFB6846FFF744FD04001022EF
:108E4000280008A902F084FB20000CB070BDF8B522
:108E500006000D0000243719AC4200D3F8BD02F023
:108E600017FB030A3B70631CDBB201379D4203D939
:108E70000234F054E4B2EEE71C00EDE773B50600EF
:108E80000C000225002819D0002917D0032101A8C1
:108E9000FFF7DDFF6B469A793F231A4001331343F6
:108EA0006A463000937101A92200FFF71BFF051EDF
:108EB00004D10322E01C01A902F08AFC280076BD3F
:108EC00003785807DA08C00FD20080009B071043D0
:108ED0009B0F1843C0B2704707230B40C908C90055
:108EE0000B4303707047000070B50400FFF7EAFE03
:108EF000134DA4006359002B21D0186A002801D01B
:108F000002F07EFC2B59986E002801D002F078FC0C
:108F10002B59D86E002801D002F072FC2B59186F23
:108F2000002801D002F06CFC2B59586F002801D0AA
:108F300002F066FC285902F063FC00232B5170BD3F
:108F40007C67FF1F0E4B8000C35870B50C00002BD0
:108F50000FD09D68002D0CD02B78201D0B706B78E6
:108F60004B70A97CFFF7B8FF2B7E23726B69E3601F
:108F700070BD10220021200002F02AFDF8E7C04653
:108F80007C67FF1F014B18607047C0467867FF1F62
:108F9000074A03008000825810B5002A06D0D08806
:108FA000984203D1012901D1FFF79EFF10BDC046B1
:108FB0007C67FF1FF0B5264E95B087000B93BB5919
:108FC0000500099112200A92002B31D0D888FFF7B2
:108FD000A5FB04001420002C2AD0280010A9FFF7BC
:108FE000B1FFBB591E781D6A002E23D00895FDF7EE
:108FF000EFFA07000020FDF7F1FA0790A379E61DCC
:10900000069310AD0CA9089800F0E2FA0EA928000A
:1090100000F0D7FA0B9B0A990493069B09980293D8
:10902000079B0396019300970EAB0CAAFFF77CFEFB
:1090300015B0F0BDFDF7CCFA06903000FDF7CEFA82
:10904000E31DA779079310AB06000893DAE7C04643
:109050007C67FF1F30B50C4C85002A59030085B092
:109060000120002A0ED018006946FFF76BFF2B592C
:109070001A78D888054B002A00D1054B6A4607218B
:1090800000F0D9FB05B030BD7C67FF1FC395001110
:10909000D195001130B5094C8500295985B01022B1
:1090A0006846253102F094FB2A591121044BD088DF
:1090B0006A4600F0C0FB05B030BDC0467C67FF1FAC
:1090C0006D96001130B5094C8500295985B01022E4
:1090D0006846353102F07CFB2A591121044BD088B7
:1090E0006A4600F0A8FB05B030BDC0467C67FF1F94
:1090F000AB960011F7B54D4F86001020F4590D00C6
:1091000002F05EFCF3592062186A132200286CD02A
:10911000033A29009C6802F05BFBF3591A7801922C
:10912000002A58D11E6A227D317B9446514001228B
:10913000019F114201D167461740217D9143394378
:109140002175377B4F40BC4660460027800701D41D
:109150004F081740012102208F40227D82433A436D
:109160002275377B5740BC4660460027400701D434
:1091700097080F400420227DBF0082433A432275A6
:10918000627D002794466046727B42400A4201D1CC
:1091900067460F400121627D8A433A436275777BBF
:1091A0005740BC4660460027800701D457080F404F
:1091B0000220627D7F00824317436775767B002221
:1091C0007E40760701D4BA080A400426617D9200E9
:1091D000B1430A4362756A78002A08D06278002A8F
:1091E00005D005220533DA7700221000FEBD0422E7
:1091F0002979114205D1A17C114202D10533033AEC
:10920000F1E7019A21782C78002A02D10A00210086
:10921000140018220429E8D8042CE6D8052060435D
:10922000034A05331218525CDDE7C0467C67FF1F16
:1092300058BD001110B50A001121024B00F0FBFAD5
:1092400010BDC046079700110B0030B587B001ADC7
:109250002B806B4604001100981D082202F0B8FA1A
:109260002A000B212000024B00F0E5FA07B030BDC8
:109270002F97001110B50A001121024B00F0DBFA04
:1092800010BDC0468397001113B50B0011006A464C
:1092900013706B4604000622581C02F099FA6A46C5
:1092A00008212000014B00F0C6FA13BDA39700115E
:1092B00010B50A001121024B00F0BDFA10BDC046E6
:1092C000F39700117FB505000B4BAA00D458080096
:1092D000002C0FD0666F237FE28821780396266FDB
:1092E0000296E66E0196A46E0094FDF709FC280034
:1092F000FFF7FAFD7FBDC0467C67FF1F10B5172141
:10930000FFF7E0FF10BD000070B50A000D00064B2E
:109310000221040000F08FFA060029782000FFF7F0
:10932000D1FF300070BDC046D396001170B586B035
:1093300000236A461370836804001D78681E0A289B
:1093400059D801A902F054FA060633373B3F434788
:109350004B4F5300180000F042F9062312284BD05F
:1093600000281BD16088FFF7D9F90823002813D003
:109370004279002A47D1264B1A78072312070BD5CA
:10938000244B1A680723002A06D01668002E03D043
:10939000290001AAB04703006A4613706B461B7888
:1093A0006088002B2AD1FFF767FC06B070BD18005B
:1093B00000F06CF9D4E7180000F087F9D0E7180046
:1093C00000F093F9CCE7180000F0ADF9C8E71800F9
:1093D00000F0C3F9C4E7180000F0F6F9C0E7180080
:1093E00000F0F6F9BCE7180000F013FAB8E718002F
:1093F00000F013FAB4E707236A46137069466088E1
:10940000FFF782FFD1E70523012AC5D1024BB8E758
:109410000966FF1F7467FF1F7867FF1FF8B52C4FA1
:109420008600F35904000D00002B40D0DA888242F8
:109430003DD15A78062A33D11A78002A2ED001203D
:1094400099681A6A097D014206D0157B054203D04E
:1094500007225A700120F8BD0220014204D0157B7A
:10946000054201D00922F4E70420014204D0127B16
:10947000024201D00B22ECE7164B1B68002BE9D00F
:109480005B68002BE6D020009847BB5900215B7831
:10949000122BDFD12000FFF715FFDBE70E4BECE7C7
:1094A000112A04D1002900D032252900F2E7002D2D
:1094B00008D12000FFF732F9002803D010230279E9
:1094C0001343037121002800FDF798FAC2E7C04654
:1094D0007C67FF1F7467FF1F7867FF1F70B50E4E14
:1094E0008500AB590400002B13D01B78002B11D141
:1094F0000A4B1B68002B04D05B68002B01D02000B6
:10950000984773595B78122B03D100212000FFF795
:10951000D9FE70BD024BECE77C67FF1F7867FF1F29
:109520007467FF1F094B8000C3581020002B0CD01C
:109530001A6A002A09D09B68002B06D0127A1B7E7B
:10954000101C9A4200D9181CC0B270477C67FF1FDC
:1095500070B503000D0014000220002A30D000294D
:109560002ED013700B78081D53704B789370FFF753
:10957000A7FCE070012002212B7A23716B7B034052
:1095800063716A7B0A401343042263716E7B164049
:10959000334363716E7BF608F600334363712B7BB4
:1095A0000340A371287B014000200B43A371297B5A
:1095B0000A401343A3712A7BD208D2001343A3713C
:1095C00070BD10B50A0001000120FFF7C1FF10BDFA
:1095D00010B50A0001000220FFF7BAFF10BD70B5F8
:1095E00006000C000220002E30D000292ED0737807
:1095F000201D0B70B3784B70F178FFF76DFC0122E2
:109600003579257271794B10080013409340104052
:109610000343881010408000C9080343C9000B436E
:109620006373B1794B10080013409340104003431B
:10963000881002409200C9081343C9000B4321203F
:109640002373FCF773FE854201D2122070BD2220E5
:10965000257AFCF76BFE8542F7D823781820042B77
:10966000F4D86378012BF1D80020EFE7030010B5A0
:109670000220002909D0002B07D00322481C0A70C1
:1096800019000D3202F0A4F8002010BD03000222E0
:10969000080010B5002B06D0002904D00E32591C4A
:1096A00002F096F80022100010BD030010B5022051
:1096B000002909D0002B07D00422481C0A70190089
:1096C0000C3202F085F8002010BD10B5FFF7DEFF68
:1096D00010BD03000220002906D0002B04D0052273
:1096E00000200A701B784B70704703000220002B8B
:1096F00008D0002906D05B7800200B70013B082BB6
:1097000000D918307047030010B50220002909D095
:10971000002B07D00622481C0A7019000A3202F0FA
:1097200057F8002010BD10B5FFF7B0FF10BD0200C4
:109730000B00022010B500290ED0002A0CD0072102
:109740001970118859701188090A99701118082226
:10975000D81C02F03DF8002010BD03000A000220D2
:1097600010B5002B0CD000290AD09978587809023E
:1097700001431180901CD91C082202F029F8002016
:1097800010BD030010B50220002909D0002B07D01E
:109790000822481C0A701900921802F019F80020DB
:1097A00010BD02000B00022010B500290BD0002ACA
:1097B00009D009211970117818185970511C062206
:1097C00002F006F8002010BD10B5FFF75FFF10BDD6
:1097D00002000B00022010B5002A09D0002907D092
:1097E0005178197011180622581C01F0F1FF002061
:1097F00010BD030010B50220002909D0002B07D0AE
:109800000A22481C0A701900063201F0E1FF00200C
:1098100010BD10B5FFF73AFF10BD02000B0002208B
:1098200010B5002A06D0002904D018005178FFF79F
:1098300053FB002010BDF0B585B017001E006A462E
:1098400006230500080091819380FEF7C0FC1324D5
:10985000011E02900CD03800B047041E05D128002C
:1098600001A9FEF76FFA041E02D0029801F058FF1A
:109870002800FFF701FA200005B0F0BDF0B50400A4
:109880008BB0019115000021102202A802F0A0F86F
:10989000334EA700B85900283CD0C388A34239D121
:1098A0000378002B36D14278062A18D10200010035
:1098B000553235310C3006ABFFF7A9FA002829D113
:1098C0002000FFF72FFE020006A902A801F080FF8A
:1098D000200002A901F0C4FD01200BB0F0BD816E93
:1098E000002917D00B8A112A28D19D420ED1019848
:1098F0001231093A01F0CCFF012807D1BB592000F1
:109900009D6EFFF70FFE29000200DEE732212000E6
:10991000FFF7D8FC2000FEF701FF061E1BD0416AAE
:10992000002918D00B8AAB4215D1082201981231B8
:1099300001F0AEFF01280ED1716A0AE09D42E9D123
:1099400008220198123101F0A3FF0128E2D1BB598E
:10995000996E8A7EB9E7200002F0AAF8BCE7C046FB
:109960007C67FF1FF0B56B4D87007E5985B033785B
:1099700002900393002B00D087E0B368346A019310
:109980007078062817D101221B7D134202D0217B5B
:10999000114218D10222134202D0217B114251D12F
:1099A0000422134203D0237B134200D08BE0019B9F
:1099B0005A7DEB5991E007380428F8D801F018FFD8
:1099C000032E42678300B36E002B03D11C2001F0ED
:1099D000F7FFB066EB599C6E002C1CD010220021C2
:1099E000200001F0F5FF0298FFF79CFD0100200028
:1099F000FFF72DFA01F04CFD2082200008211230E3
:109A0000FFF725FA0298FFF78DFDA076EB592100AC
:109A1000D888FFF70FFC0822EB591CE0B36E002B2F
:109A200005D01A00198AF0881232FFF70DFC0222C5
:109A3000019B197DEB5911423DD0207B10423AD059
:109A4000073208E0F488FCF7DBFD01002000FFF797
:109A500011FC0A22EB595A70029B9C002A59537838
:109A6000073B042B11D8D088FEF758FE00284ED0B3
:109A7000C3895A08D2182849029B0298CB542B5903
:109A800041180433254801F02BFF05B0F0BDFCF769
:109A90009FFD03000120834201D100200393EB5975
:109AA000DE88FCF79BFD039902003000FFF7ECFB1A
:109AB000019AEB59117D042211420CD0217B1142F5
:109AC00009D00B22C7E7F688FCF73CFD0100300007
:109AD000FFF7EEFB6BE7019A527D01210A4204D0A9
:109AE000607B084201D00C22B5E702210A4204D073
:109AF000607B084201D00E22ADE704210A4204D067
:109B0000627B0A4201D01022A5E71222A3E7FA22C3
:109B10005200B0E77C67FF1F8067FF1FDB9E0011CC
:109B200010B5064B1A780423100018401A4200D0D2
:109B30000348FFF727FA002010BDC0460966FF1F43
:109B40008C44FF1F70B50400FFF7D4FA051E43D103
:109B50002000FFF77FFA234EA400A0598268937C6F
:109B6000DB0708D50321036A1B790B40012B02D1C7
:109B7000017F0B430377431DD97F8B1E022B0DD82A
:109B8000022900D00121C088FCF790FF042133593D
:109B90001A7F59700A431A77280070BD01290CD129
:109BA00002231022437000210C3001F011FF3059C4
:109BB00010213530FFF74BF9EEE70529ECD10223F0
:109BC000D118437010220C3001F002FE04233259E8
:109BD000117F0B431377EAE708251828DCD1053DF0
:109BE000DAE7C0467C67FF1FF0B58BB0059143886C
:109BF0007E4F9E00F45915000493002C15D10129C5
:109C000002D000200BB0F0BD101D57781678FFF77A
:109C100057F9EB68320002932B7A04990193009074
:109C20003B002000FCF70CFFEBE7E388049A93422B
:109C300001D00820E6E72378012B00D1D4E0059B72
:109C4000581E092800D9CFE001F0D2FD05CE0A291F
:109C5000CC506C859AB229000498FFF773FFD1E7C6
:109C6000200029001022453001F0B2FDB9594B788F
:109C7000042B02D1013B4B70C3E70B000A002533D4
:109C800035320C310498FFF795F90498FFF702FA82
:109C90000522431E9841BB59C0005A70B2E720000C
:109CA00029001022553001F093FD049B4F4C9D007C
:109CB000295904980A0006AB55320C31FFF77AF99E
:109CC00029591022453106A801F0E2FD012808D1EA
:109CD0000498FFF7F7F90590002804D106222B59C4
:109CE0005A7005988EE708230593FAE763780C2BE2
:109CF0007AD1E36E002B03D11C2001F061FEE066F7
:109D0000BB59D86E00286FD01022290001F060FDE9
:109D1000BB590498DC6EFFF705FC0D22A076BB59F9
:109D20005A706EE7E06E00285ED063780D2B5BD131
:109D30002B8808220382A91C123001F049FDBB596F
:109D40009A68517D0222114226D0186A407B104247
:109D500022D00C32E4E763780E2B45D1236F002B21
:109D600003D1162001F02CFE2067BB59186F002884
:109D700003D01022290001F02BFD0F22BB59CFE7A1
:109D800063780F2B30D1206F0622691C103001F050
:109D90001FFDBB599A68517D0422114203D0196AF4
:109DA000497B1142D5D100210498FFF78BFA28E7AF
:109DB000636F002B0DD0BB59586F0028F3D01022D1
:109DC000290001F005FD0122BB5952425B6F1A6167
:109DD000E9E7142001F0F4FDBB5960675B6F002BCD
:109DE000E9D126E72978DFE707200BE77C67FF1F2B
:109DF00010B5064C207001F04BFC06212078FDF7D1
:109E000091FF0348FEF778FC10BDC0468F67FF1F27
:109E1000918F001100200BB270B50D00834216DA4D
:109E2000264B187801F09CFC041E0DD00378922B71
:109E30000ED0A02B37D0224B1878FF283AD0210023
:109E400001F0AEFC002835D180200002684070BDD2
:109E500043780E2B0BD03E2BEDD18378052B12D0FF
:109E6000082BE8D181798088FFF7D8FA08E0154BF4
:109E700082889A42DFD183681878591CFEF7C0FEA9
:109E8000002817D1D7E7104B1B785B0712D50F4B73
:109E90001B68002B0ED09B68002B0BD0C289811D44
:109EA00080889847ECE7FFF741FAA068002801D0C6
:109EB00001F036FC200001F063FDC5E78F67FF1F4E
:109EC0008544FF1F182000000966FF1F7867FF1FE9
:109ED00010B50078FFF712FA10BD10B50078FFF743
:109EE000FDFA10BD0C234343084A10B59B185A686D
:109EF000002A03D0012901D1904710BD9B68002B97
:109F0000FBD00029F9D19847F7E7C046AC67FF1F9F
:109F100010B5162813D801238340094A946B1C43BB
:109F20009463506B98435063D46B2000984301298D
:109F300001D120001843D063116B0B43136310BD94
:109F400000800040F0B500240127154B85B0DA6B86
:109F5000144E03921A6C0192DA64019BE3403B4277
:109F600017D0039DE5403D400295E5B202992800D7
:109F7000FFF7B8FF316A736A002908D03900002B57
:109F800001D0029979402800FFF7C2FF01E0002BC1
:109F9000F9D101340C36172CDFD105B0F0BDC04625
:109FA000008000409067FF1F10B5012402002000D0
:109FB000162A08D8054B5968D140214204D01868A8
:109FC000D0400123184010BD186DF9E70080004013
:109FD000162807D80122064B8240002903D0D968F1
:109FE0000A43DA607047D9689143D960FAE7C046FE
:109FF0000038004030B5162818D8032444430F4BCE
:10A00000E25C1B199C785D7801232D1B0135AB4068
:10A01000013BA340A140DB430C00122807D80849AC
:10A0200092005218116819402143116030BD054A51
:10A0300011680B4023431360F8E7C0469FBD001131
:10A0400008F0004014F00040C21F70B5D4B20623DF
:10A05000092C0BD80125084C9540002908D0002177
:10A06000FFF7C8FF23682B4323600023180070BD4F
:10A070002368AB43F8E7C04600380040F0B5162827
:10A0800026D8214B1B185B78022B21D10324444393
:10A090001E4A1F4EA35C12199478012215008540B8
:10A0A000B76B013CE4B23D43A240B563194C1228A2
:10A0B00015D89B0000290CD117495B1899680A43F1
:10A0C0009A600123205C154A834011680B4313609A
:10A0D000F0BD11495B18996891439960F1E70E4B07
:10A0E00000290DD159690A435A61225C1328E8D02E
:10A0F0000123203A93400A49086803430B60E7E7CD
:10A10000596991435961F0E79067FF1F9FBD0011A6
:10A1100000800040E4BD001100F00040A0F00040CD
:10A12000A4F00040F8B500241B4E1C4D1C4B1B5DD9
:10A13000012B1FD1184A9269E2401A420BD001222A
:10A14000AA5693402200143AD2B2022A09D81549DD
:10A150004A6913434B6101340C360235172CE5D1A3
:10A16000F8BD0022AA560F499200521891680B437D
:10A170009360F0E7022BEED1E7B23800FFF714FF4F
:10A1800001235840C1B23800FFF778FF3800FFF7CD
:10A190000BFF7077DFE7C0469067FF1F71BD0011AE
:10A1A0009167FF1F00F00040012202388240054BFA
:10A1B000002903D059690A435A617047596991438C
:10A1C0005961FAE70038004070B504000D00052021
:10A1D000162C1AD800212000FFF7FAFEA31E012B2F
:10A1E00003D801212000FFF7DFFF00212000FFF747
:10A1F0002BFF01220A49A2400A4B4868012D05D1D4
:10A2000002431B194A605D70002070BD9043486096
:10A2100002211C196170996991439961F4E7C04664
:10A22000008000409067FF1F10B516280AD8012251
:10A23000074B8240002906D019680A431A600121A1
:10A24000FFF7C2FF10BD196891431960F7E7C046D8
:10A250000080004070B505000520162D17D80C238E
:10A2600000246B430A4A21009B181C70094B2800EC
:10A270005B195C70FFF7A8FF0123AB402000064983
:10A280000A681A430A6005490A689A430A6070BD61
:10A29000AC67FF1F9067FF1F348000403080004094
:10A2A00070B504000E00FF2813D003250540FFF70A
:10A2B000D1FF084AA3089B009B183F22ED00AA404B
:10A2C000AE40196820009143314319600121FFF726
:10A2D0007FFE70BD18380040F8B505000520162D2A
:10A2E00025D80C246C43124BE4186368002B03D16F
:10A2F000A3680D30002B1AD0022201270D4B00213C
:10A300005B195A7028002770FFF75EFF63681E1EF6
:10A3100008D0A3683E00002B04D02800FFF744FEBD
:10A320004640F6B228003100FFF7F2FD0020F8BDEC
:10A33000AC67FF1F9067FF1FF7B5C420FF222B4BB0
:10A3400080001958002491437F3A0A431A50802212
:10A35000274F5202274E1A60274B1D5D002D21D03A
:10A36000A31E012B03D80121E0B2FFF71DFF012D31
:10A3700018D11F4B9B69E3402B4213D0E3B2180066
:10A380000193FFF711FE01000198FFF74DFFE3B2C3
:10A39000143B022B1DD801217156184A8D40536978
:10A3A000AB4353613B7F002B0DD0E5B22800FFF794
:10A3B00093FF2800FFF7F8FD7B7F0100834202D066
:10A3C0002800FFF78FFD01340C370236172CC3D15C
:10A3D000F7BD012100237156F3568D40074A9B00BB
:10A3E0009B189A68AA439A60DCE7C04600E100E047
:10A3F0009067FF1F71BD00119167FF1F00F00040C3
:10A4000010B504000520162C0CD801212000FFF700
:10A41000DBFE0123044A002011194B70A34091690F
:10A420000B43936110BDC0469067FF1F70B50E00CF
:10A4300015000400FFF70EFF0C236343094A2000B8
:10A440009B189D605E60FFF747FFF021064B074AAF
:10A450008900051E5A5002D02000FFF7FBFE28009D
:10A4600070BDC046AC67FF1F0000FF1F459F001175
:10A4700070B5134D07202C78002C1FD19822210095
:10A480005200280001F004FB0123C420FF222B709E
:10A490000C4B80001C635C630B4B1C605C600B4BC3
:10A4A000195891437F3A0A431A50802252021A6087
:10A4B0000D20074A074901F0BBF9200070BDC046D6
:10A4C0009067FF1F00800040A0F0004000E100E026
:10A4D00039A3001125A10011030010B50620072B98
:10A4E00009D8054A137001F0F3F8D7210020034B77
:10A4F000034A89005A5010BDB444FF1F0000FF1FDB
:10A50000151BFF1F70B51D0002240C2910D8094A25
:10A51000CA40D2070CD5FBF715FF041E08D1059AD7
:10A5200004992800FBF72AFFFCF798FDFFF7F8FADB
:10A53000200070BD1210000030B50D7802232C00F1
:10A540009C43184201D02B431C0008252300AB4339
:10A55000284201D02B00234320241D00A543204284
:10A5600001D01C4325002A230D70184204D0117815
:10A570001E3B0B43137030BD0028FCD10C21137817
:10A580008B43F7E7F8B51D0006AB1B88140007AA3C
:10A590000E000B201778002B27D10A78022A49D108
:10A5A0004A68507811780002244A08438018042829
:10A5B00040D801F01DF903121D1B2300F06801F0C3
:10A5C0006FF9021CC0B2B84200D93A1CD2B22000C6
:10A5D000F1682A8001F0FCF806E00222F3681B888B
:10A5E0002A8023701B0A63700020F8BD0622EEE764
:10A5F00001232B80F3681B782370F5E7F368002BA9
:10A6000016D008222A801A8822701A88120A6270CC
:10A610005A88A2705A88120AE2709A8822719A881F
:10A62000120A6271DA88A271DB881B0AE371DBE728
:10A630002B80D9E701202B80D7E7C04600D6FFFF4B
:10A64000F7B516000A781D0008AB1F880C0001231F
:10A65000022A18D14A685078117800022B4A084320
:10A66000801803280FD801F0C3F802254439E068A8
:10A6700001F016F9C0B20723B84204D37B19019345
:10A68000152B02DD0D231800FEBDE0682A00310005
:10A69000C01901F09DF86B4600209B88E268D054F9
:10A6A0001B4B1B68834203D01B68834200D0984732
:10A6B0000023E8E70B23002FE5D1022DE2D17378C8
:10A6C00032781B021343E2681380114B1B68002B86
:10A6D000EED01B68002BEBD00120E8E70B23002F06
:10A6E000D1D1062DCED12A003100E06801F070F8FA
:10A6F000DEE70B23002FC6D1012DC3D1327875338D
:10A70000012AC0D8E3681A70D2E7C04600D6FFFF1E
:10A710009C69FF1F70B50C001500072837D801F0A1
:10A7200067F8041436361B36242E182015290BD84A
:10A73000184E16220021300001F04AF922002900AB
:10A74000300001F045F8002070BD18200229FBD12F
:10A750001288114B1A80F6E718200829F4D10A0054
:10A760000E48290000F0ECFFEDE718200129EBD19D
:10A770000B4B10780B49DA69FFF7DEFEE3E7182090
:10A780000129E1D1064B10780749DA6BF4E7022082
:10A79000DAE7C0468469FF1F3245FF1F2845FF1FC7
:10A7A000B844FF1FE044FF1F0045FF1F030010B522
:10A7B0000020DB0704D50721024A034800F08CF88B
:10A7C00010BDC046FCBD0011B844FF1F054A030080
:10A7D0001068002803D082889A4201D180687047AF
:10A7E0000068F6E7A06BFF1F0A88030008009A4282
:10A7F00004D08A8804309A4200D0002070470000BC
:10A80000F8B5F82200230D4F0D4E7968050042433C
:10A810003370994200D07B600A4C0021200001F087
:10A82000D7F800231A007C60AB4202D100203370BD
:10A83000F8BD01332280DBB2F834F5E7A06CFF1FCE
:10A840009C6CFF1FA46BFF1F73B56B460190060045
:10A85000684615001980FCF733FF041E11D1002D46
:10A860000FD07689002E11D00C2001F0A9F8002815
:10A870000ED0084A0460136886808560002B02D1E0
:10A880001060200076BD1A001B68F7E70224F8E785
:10A890001324F6E7A06BFF1F012100220A4B10B51D
:10A8A00049420A4C198099809A719A70084B20701D
:10A8B000012019805A60FFF7A3FF2078FCF75EFFA4
:10A8C0000448FDF719FF10BDA469FF1FA86CFF1F06
:10A8D000A06CFF1F85A90011022310B5002802D02B
:10A8E000FFF7B2FF0300180010BD0000030010B511
:10A8F0000020DB0704D50421024A0348FFF7A4FF28
:10A9000010BDC04610BE00113845FF1FF0B50E2621
:10A9100087B003930CAB1F8802ABF6180500080044
:10A9200031000292FDF74EF804000120002C0FD0F8
:10A930003088FFF74BFF03000E20002B08D05E6825
:10A94000002E05D021002800039B029A0097B047F3
:10A9500007B0F0BD0A4B10B5984207D10122002381
:10A9600052420A808B708A808B7110BDFFF73CFFCA
:10A970000028FAD001235B42038000238370F4E7B0
:10A98000FFFF0000F8B5050001290AD1134E00248D
:10A990003388F827AB4219D028001149FFF7DAFFB6
:10A9A00006E0022904D10139FDF724FF0028EDD08B
:10A9B000F8BD3B0063437268D018D35A002B09D00E
:10A9C0003A00002101F004F80134E4B2054B1B7891
:10A9D000A342EED801235B423380DDE7A06CFF1F6A
:10A9E000A469FF1F9C6CFF1F10B5FFF7FDFE03005D
:10A9F0000020834200D0987810BD0000F0B589B0E7
:10AA00001C000EAB80CB03901E8810AB1B78049209
:10AA100002930B7A0D00DB0616D42B780593022BDC
:10AA200024D00498FFF7D2FE002812D003689C4679
:10AA3000002B0ED0029B2200019329003B006446AC
:10AA400003980096A04705E00498FFF7BFFE002892
:10AA500002D10E2009B0F0BD8368002BF9D00A2284
:10AA60002900039898470028D7D0F3E76B685878F7
:10AA70001A786B4B000210439842D2D8043B98429C
:10AA800010D2684B984242D015D8674BC0180128A5
:10AA9000C7D80B20002EDDD1EB681A7859683A80B0
:10AAA000200028E0614BC018032800D979E000F0AD
:10AAB0009FFE846A789E5E4B9842B2D10B20002E96
:10AAC000C8D101233B80EB6831001B782370688973
:10AAD000013080B2FCF776FF3A88031E0ED0017871
:10AAE00002328A183A80428962704289120AA27040
:10AAF00059680278E01C00F06BFE06E004323A80F0
:10AB000031000422601C00F063FF0020A2E70B204C
:10AB1000002E9FD1EB6807A91E8804233B80330ACF
:10AB2000300026706370FCF74DFF051E28D004AB83
:10AB30009A890E2304A95B183E49C668FCF7B6FF44
:10AB400000280BD12B783C486A680599FBF76CFB11
:10AB5000002803D1012304AA5B42D3813278022A60
:10AB600006D17168201D00F033FE3B8802333B8024
:10AB70000E2304AA9B181B88A3701B0AE370C4E76A
:10AB800004ABDE81F4E70B20002E00D062E7E96819
:10AB90000398FFF729FF02233B802070000A6070B2
:10ABA000B3E70B20002E00D054E70222EB681B888D
:10ABB0003A8023701B0A6370A7E7E86800F070FE14
:10ABC000C2B203000720B24200D243E70DD002997F
:10ABD000DBB27118994202DB921BD3B20293029B43
:10ABE000E9681A003B8089195AE70023F6E70B2031
:10ABF000002E00D02EE70722EB683A801A782270E8
:10AC00005A7862705A88A2705A88120AE2701A79C9
:10AC10002271DA886271DB881B0AA37175E7C0466E
:10AC2000042900000228000000D8FFFFFFD6FFFF24
:10AC300003280000FFFF000040BD0011F0B58DB0FB
:10AC40006B460020089120229B5E83423DDAA64B92
:10AC5000187800F085FD071E32D00378B02B2CD178
:10AC60000079023816281FD800F0EAFD17001E00F0
:10AC70001E001E0031001E0096001E001D011E0059
:10AC800052011E0073011E00CD011E0050021E0065
:10AC90001E001E008E021E00E302944B94491B8886
:10ACA00078880B80FBF700F83800FCF781FF914BA8
:10ACB0001B68002B01D038009847380000F060FE78
:10ACC0008020089B0002434018000DB0F0BDF62222
:10ACD0000021874800F07CFE0BAA3B7B79893889EC
:10ACE00000923A000D32FCF785FD0400804B1B7882
:10ACF000002C3FD146E0804B788805937F4B410084
:10AD0000CB5A0BAE073BDBB2328802930023019390
:10AD10007B4B210006930093059BFFF76FFE744D5C
:10AD2000002810D1069B3A8A1B889A420BD1380022
:10AD30000599123000F0ACFD002804D02B78628910
:10AD40009B00EB185A80162306A81B183288200097
:10AD50007989FCF7ABFE2B7804009A00AA18518879
:10AD60000029C3D00133DBB22B70002807D006A91D
:10AD7000C98A9180634A12889A42BCD802E00121B4
:10AD800049429180002B04D059497888FAF7C0FFD6
:10AD90008AE73E890A2479E000253E89574B0693CD
:10ADA0007B88069A5B009B5A033B9D4202DB002D89
:10ADB000F0D05BE0162206A812183B7B798900923E
:10ADC0003A0030000D32FCF715FD0590002858D0F0
:10ADD0004689017A7888FCF7D7FC041E44D1464B9B
:10ADE00078880793069B4100C95A454B0439C9B27C
:10ADF00006AAD28A06930291019400930599079BB3
:10AE0000FFF7FCFD041E2FD1069B39491A88931CBD
:10AE1000002D26D14B807988384B4900CB5A5119E7
:10AE2000033B8B4220DD059B31485B8941190B7147
:10AE3000A91C0135C9B2EDB2059145191B0A2B7148
:10AE4000059B2D490433181800F0C2FC2C4B059AC1
:10AE50001B88D318DDB22C4B9E4205D00136B6B20A
:10AE60009CE749889942D6D0002D0CD0204C280070
:10AE7000618800F0D5FA207021007888FAF758FF31
:10AE800012E7059CF0E7002C00D183E77B78142BB8
:10AE900000D109E716493B794E800B700C71788818
:10AEA000FAF7F8FE00E7162406ABE418210038890B
:10AEB000FCF788FD011E00D1B7E1788822880F4C8D
:10AEC00045002C5B0A4D013CE4B2029400240F4B78
:10AED00001940095FFF792FD041E00D014E12900B3
:10AEE0007888FAF735FFDFE6A86CFF1F2444FF1FC0
:10AEF000AC69FF1FA069FF1FA66AFF1FDC65FF1F6B
:10AF00009C6BFF1F2244FF1FFFFF0000AE69FF1F65
:10AF1000162406ABE41821003889FCF753FD011E06
:10AF200000D182E178882288AE4C45002C5BAE4D82
:10AF3000013CE4B202947C89AC4B01940095FFF78C
:10AF40005DFD041E00D0DFE029007888FAF70AFFD3
:10AF5000AAE60025A44B1D803B00FE331B78A24AC5
:10AF600078880792AB4208D99E4B128806930699BF
:10AF700043005B5A013B9A4203DB0799FAF7FCFE58
:10AF800092E616246B00FB18059306ABE418059BAC
:10AF900021001889FCF716FD011E03D1059B012431
:10AFA0001E8973E77888924B2288069C0993430098
:10AFB0001B5B904E013BDBB2029300230096019392
:10AFC000099BFFF71BFD041E02D0059B1E895DE750
:10AFD0007B88069A5B009B5A079A10883288121861
:10AFE000934202DC1B1A013B33807F4C02303288D3
:10AFF0000999001900F0ECFB2388328801359B1871
:10B000002380EDB2A8E70BAA3B7B798938890092AF
:10B010003A000D32FCF7EEFB00250590059B002B56
:10B0200004D10A24002D00D16EE060E0059B7888F1
:10B03000197AFCF7A9FB0100041E63D1694C6C4B23
:10B04000788806940993069B4400E45A694B063CB1
:10B05000E4B20BAE328807930294019100930599F4
:10B06000099BFFF7CBFC041E4CD1079B5E491B8854
:10B070001A1D002D30D14A80059B5B4C5A896319FB
:10B080001A716B1C9BB2E318120A1A71162306A8D8
:10B0900032881B1879890598FCF708FDFF21AA1C46
:10B0A0002E1D03350B00059092B2B6B2ADB200284A
:10B0B00003D006ABDB8AD9B21B0AA218651911713D
:10B0C0002B714C4D301D2A884949201800F080FB17
:10B0D0002B88F618B5B2A1E74988914207D17A8842
:10B0E00006995200525AEB18053A9A42C4DC3E4C7B
:10B0F0002800618800F02CFC207021007888FAF785
:10B1000045FED1E5002DF2D13E89BFE6162606ABFD
:10B11000F61831003889FCF755FC3D000400FF3576
:10B1200000282DD0037A9B060CD400227B89398914
:10B13000788800923A000C32FFF7E8FB041E10D02A
:10B140003E8915E03088FFF741FB00281AD083685C
:10B15000002B17D02100122278889847041EE4D0D3
:10B16000EEE7AB78002B02D17888FAF71FFE0026B5
:10B17000AB78002B00D097E5002C00D194E585E654
:10B180000124DDE70E24DBE7162506ABED182900C8
:10B190003889FCF717FC041E47D0037A9B0611D4AC
:10B1A000154A7B881188994203D01448814207D1FF
:10B1B0001380134BF8261D780023D9B2A94221D35E
:10B1C0000924A1E72888FFF701FB00282FD0836816
:10B1D000002B2CD02100122278889847041EDFD043
:10B1E00092E7C046DC65FF1FAC69FF1FAE69FF1F19
:10B1F000A66AFF1F9C6BFF1FA06CFF1FFFFF0000D4
:10B200009C6CFF1F31005943546801336018615A28
:10B210000029D2D13C0008342100F82200F0D8FAED
:10B2200021007888FAF7CAFD3EE501246CE70E2478
:10B230006AE71D4B1A887B889A4231D07888FAF7E2
:10B24000C7FD31E5F823059851684343CD18C95A25
:10B2500000291FD03B7A012B0BD16C88AB887888F2
:10B26000AA1D0094FFF752FB041E02D000233B727C
:10B270002E88F8220021280000F0AAFB00232B8052
:10B28000059B0133DBB20593084B05991B78064AF1
:10B290008B42D7D801235B421380002CCED0F5E53A
:10B2A000002634000596EFE7A06CFF1F9C6CFF1F83
:10B2B00070B504000E001500FFF796FA031E08D1C2
:10B2C00031000548FFF790FA03001120002B02D04F
:10B2D0001C8000209D7070BDFFFF0000F8B50B4F73
:10B2E00006003B780D001400FF2B0ED00A2000F062
:10B2F00067FA011E09D0B123038000234680037141
:10B30000C5800481387800F04BFAF8BD7945FF1FFD
:10B31000F7B50F0008A90600088809A90B240988B9
:10B32000002821D10234022B1ED1557813782D022A
:10B330001D432B008B4301937334002B14D1FB6806
:10B34000300019000093FFF74FFB019C85420BD0A2
:10B350002A0030000099FFF7ABFF041E04D12A0039
:10B3600030007989FFF7BAFF2000FEBDF0B50E78F6
:10B3700085B003900AA805880120022E0DD14C68E3
:10B380002778647824023C43054FBC4205D10398DA
:10B39000DBB201960095FFF7BBFF05B0F0BDC046DC
:10B3A0000229000010B504000C4800F061F80C48B8
:10B3B000A16B00F05DF80B48E16B00F059F80A480A
:10B3C000216C00F055F8094B0948196800F050F855
:10B3D000084B1B68002B00D09847FEE7F6BB001116
:10B3E0000CBC00111BBC00112ABC001104ED00E0D4
:10B3F00039BC0011AC6CFF1F002307B501A80193F5
:10B40000FFF7D0FF044A0548002110B5121A00F0DA
:10B41000DFFAF8F7D1FAFEE7B06CFF1F7C45FF1F9B
:10B4200001B40248844601BC604700BF350E0000ED
:10B4300001B40248844601BC604700BF291C0000DB
:10B4400001B40248844601BC604700BF5147010077
:10B4500001B40248844601BC604700BFADAE0000A5
:10B4600001B40248844601BC604700BF311B0000A4
:10B4700001B40248844601BC604700BFE53A0100C0
:10B4800001B40248844601BC604700BFB54C0100CE
:10B4900001B40248844601BC604700BF2951010045
:10B4A00001B40248844601BC604700BF9135FF1FCC
:10B4B00001B40248844601BC604700BF090E000089
:10B4C00001B40248844601BC604700BFC94A01007C
:10B4D00001B40248844601BC604700BF35550000F6
:10B4E00001B40248844601BC604700BF353BFF1FE2
:10B4F00001B40248844601BC604700BF691F0000D8
:10B5000001B40248844601BC604700BF4134FF1FBC
:10B5100001B40248844601BC604700BF6939FF1F7F
:10B5200001B40248844601BC604700BF6932FF1F76
:10B5300001B40248844601BC604700BFDD30FF1FF4
:10B5400001B40248844601BC604700BF75A90000F1
:10B5500001B40248844601BC604700BF4551010068
:10B5600001B40248844601BC604700BFA54F0100FA
:10B5700001B40248844601BC604700BF9130FF1F00
:10B5800001B40248844601BC604700BFC132FF1FBE
:10B5900001B40248844601BC604700BF055E00005C
:10B5A00001B40248844601BC604700BF8B520100D1
:10B5B00001B40248844601BC604700BFE92800008E
:10B5C00001B40248844601BC604700BF8132FF1FBE
:10B5D00001B40248844601BC604700BF3D1800002A
:10B5E00001B40248844601BC604700BF55220000F8
:10B5F00001B40248844601BC604700BF5539FF1FB3
:10B6000001B40248844601BC604700BFB352010048
:10B6100001B40248844601BC604700BF9938FF1F4F
:10B6200001B40248844601BC604700BFE117000036
:10B6300001B40248844601BC604700BFF94C0100D8
:10B6400001B40248844601BC604700BF7D18FF1F5B
:10B6500001B40248844601BC604700BFD91B00000A
:10B6600001B40248844601BC604700BFF30E0000ED
:10B6700001B40248844601BC604700BF456B01002D
:10B6800001B40248844601BC604700BF1D4B010065
:10B6900001B40248844601BC604700BFC9260000CF
:10B6A00001B40248844601BC604700BFA139FF1FB6
:10B6B00001B40248844601BC604700BFE139FF1F66
:10B6C00001B40248844601BC604700BF0134FF1F3B
:10B6D00001B40248844601BC604700BF151BFF1F30
:10B6E00001B40248844601BC604700BF8552010096
:10B6F00001B40248844601BC604700BF017F0000DE
:10B7000001B40248844601BC604700BF21460100E5
:10B7100001B40248844601BC604700BF6571010066
:10B7200001B40248844601BC604700BFD94901000A
:10B7300001B40248844601BC604700BFC9A90000AB
:10B7400001B40248844601BC604700BF810E00007E
:10B7500001B40248844601BC604700BF9DA90000B7
:10B7600001B40248844601BC604700BFF54E0100A9
:10B7700001B40248844601BC604700BFD1A5000067
:10B7800001B40248844601BC604700BF8D3AFF1FE8
:10B7900001B40248844601BC604700BFB14E0000BE
:10B7A00001B40248844601BC604700BF594F010004
:10B7B00001B40248844601BC604700BFEDA500000B
:10B7C00001B40248844601BC604700BF1D4D010022
:10B7D00001B40248844601BC604700BFE94C010047
:10B7E00001B40248844601BC604700BF4D1F000001
:10B7F00001B40248844601BC604700BF453CFF1FBE
:10B8000001B40248844601BC604700BF014C0100FE
:10B8100001B40248844601BC604700BFC95C010016
:10B8200001B40248844601BC604700BFE5480000FF
:10B8300001B40248844601BC604700BF0933FF1FC2
:10B8400001B40248844601BC604700BF593CFF1F59
:10B8500001B40248844601BC604700BF093BFF1F9A
:10B8600001B40248844601BC604700BF21240000A7
:10B8700001B40248844601BC604700BF5952010030
:10B8800001B40248844601BC604700BF8D1200002D
:10B8900001B40248844601BC604700BFCD4C0100A2
:10B8A00001B40248844601BC604700BFDD5201007C
:10B8B00001B40248844601BC604700BF0189000012
:10B8C00001B40248844601BC604700BF5118FF1F05
:10B8D00001B40248844601BC604700BF6DBC000053
:10B8E00001B40248844601BC604700BFA94601007C
:10B8F00001B40248844601BC604700BFC51D00007A
:10B9000001B40248844601BC604700BFA134FF1F58
:10B9100001B40248844601BC604700BFF136FF1FF6
:10B9200001B40248844601BC604700BF4550000096
:10B9300001B40248844601BC604700BF213AFF1FA2
:10B9400001B40248844601BC604700BF25260000C0
:10B9500001B40248844601BC604700BF090E0000E4
:10B9600001B40248844601BC604700BF851F000047
:10B9700001B40248844601BC604700BF350E000098
:10B9800001B40248844601BC604700BF434D01003A
:10B9900001B40248844601BC604700BFC53F0000B7
:10B9A00001B40248844601BC604700BF313CFF1F20
:10B9B00001B40248844601BC604700BF056A00002C
:10B9C00001B40248844601BC604700BF3D4B010002
:10B9D00001B40248844601BC604700BF154D010018
:10B9E00001B40248844601BC604700BFED4A010033
:10B9F00001B40248844601BC604700BFC56D010028
:10BA000001B40248844601BC604700BFC521000064
:10BA100001B40248844601BC604700BF1537FF1FD0
:10BA200001B40248844601BC604700BF0124000005
:10BA300001B40248844601BC604700BF5D170000A6
:10BA400001B40248844601BC604700BF5125000094
:10BA500001B40248844601BC604700BFE537FF1FC0
:10BA600001B40248844601BC604700BF554901004B
:10BA700001B40248844601BC604700BF0D5201007A
:10BA800001B40248844601BC604700BF7918000039
:10BA900001B40248844601BC604700BFB70E0000F5
:10BAA00001B40248844601BC604700BF1147010051
:10BAB00001B40248844601BC604700BF091B000076
:10BAC0000002010302020303040305020602070247
:10BAD000080209030A030B030C020D020E030F03F5
:10BAE000100311031303140315001600793D001110
:10BAF000AD3D0011000000000200000002BB00117B
:10BB0000192A0F180A000000F1590000FD24000056
:10BB100041460100017E0011159E0011697200115D
:10BB2000057C0011995100113DAC0011554E0011DA
:10BB3000713F0011A1400011000000001616000026
:10BB4000020000004CBB0011F4FFF3FFD2FC000028
:10BB50005D41001100000000000000005475796193
:10BB60000056302E37003030303100676974687508
:10BB7000622E636F6D2F70767678005448303500F2
:10BB80000200000094BB0011292A282A272A262A0D
:10BB9000252A242A0A180000E2040000710200008D
:10BBA00078EC0000744000001027000060F00000F6
:10BBB00006640000204E00000000000000000000AD
:10BBC0001F501D00023C020000011500070000008C
:10BBD000A302000030313233343536373839414230
:10BBE00043444546005048592B36325858504C551E
:10BBF0005330353034005B48617264206661756C87
:10BC0000742068616E646C65725D0A004C5220207D
:10BC1000203D203078253038780A005043202020FD
:10BC20003D203078253038780A0050535220203D8E
:10BC3000203078253038780A0049435352203D207F
:10BC40003078253038780A00A9550011FD550011CB
:10BC5000000000000200000060BC00116F2A6E2A84
:10BC60001A18D880F060FFFFFFFFFFFFFFFFFFF310
:10BC700003B59747D6F613F7D777E6F0A7F4740025
:10BC8000000001A0000000006410B71DC8206E3B3A
:10BC9000AC30D9269041DC76F4516B6B5861B24DD3
:10BCA0003C7105502083B8ED44930FF0E8A3D6D63D
:10BCB0008CB361CBB0C2649BD4D2D38678E20AA0A5
:10BCC0001CF2BDBDFB349B5F8000008000100000B3
:10BCD000000000006B5E0011F57400118F5E001112
:10BCE000FD780011135F0011D3780011895F0011F6
:10BCF000A9780011DB5F0011717A00114360001117
:10BD0000717A0011756000112B7A0011895F0011A2
:10BD10006178001101600011097A00110000000033
:10BD200000000000E7600011097A0011496100116C
:10BD30000D750011052A042A012A002A0229032868
:10BD40000128002801180018000000000000000071
:10BD50000000000000000087010102010201010251
:10BD600001020303040103010101010103030201B4
:10BD700003000D000E001000110013001401070154
:10BD800008010A010B011C011D0204020502070241
:10BD9000080219021A021C021D0301030203170004
:10BDA0000201000504000807000B0A001716001D19
:10BDB0001C010201010504010E0D011110011413F3
:10BDC000011716011A19020201020B0A020E0D02D6
:10BDD0001110021413021716030504030807030BBE
:10BDE0000A030E0D0001020307090A0B0E0F1011C2
:10BDF00012141718191A1B1F2021220085A50011E3
:10BE000041A60011000000000200000046BD001124
:10BE1000000000006DB300110000000002000000EF
:04BE200044BD00110C
:020000041FFFDC
:1000000000000000D53E001108BB001104BB001128
:100010008862FF1F000000000000000000000000D8
:1000200000000000000000000000000000000000D0
:1000300000000000000000000000000000000000C0
:1000400000000000000000000000000000000000B0
:1000500000000000000000000000000000000000A0
:100060000000000000000000000000000000000090
:100070000000000000000000000000000000000080
:100080000000000000000000000000000000000070
:100090000000000000000000000000000000000060
:1000A0000000000000000000000000000000000050
:1000B0000000000000000000000000000000000040
:1000C0000000000000000000000000000000000030
:1000D0000000000000000000000000000000000020
:1000E0000000000000000000000000000000000010
:1000F0000000000000000000000000000000000000
:1001000000000000000000000000000000000000EF
:1001100000000000000000000000000000000000DF
:1001200000000000000000000000000000000000CF
:1001300000000000000000000000000000000000BF
:1001400000000000000000000000000000000000AF
:10015000000000000000000000000000000000009F
:10016000000000000000000000000000000000008F
:10017000000000000000000000000000000000007F
:10018000000000000000000000000000000000006F
:100190006534FF1F5533FF1FC166010000000000DA
:1001A000000000000000000000000000000000004F
:1001B000000000000000000000000000000000003F
:1001C000000000000000000000000000000000002F
:1001D000000000000000000000000000000000001F
:1001E000000000000000000000000000000000000F
:1001F00000000000000000000000000000000000FF
:1002000000000000000000000000000000000000EE
:1002100000000000000000000000000000000000DE
:1002200000000000000000000000000000000000CE
:1002300000000000000000000000000000000000BE
:1002400000000000000000000000000000000000AE
:10025000000000000000000000000000000000009E
:10026000000000000000000000000000000000008E
:10027000000000000000000000000000000000007E
:10028000000000000000000000000000000000006E
:10029000000000000000000000000000000000005E
:1002A000000000000000000000000000000000004E
:1002B000000000000000000000000000000000003E
:1002C000000000000000000000000000000000002E
:1002D000000000000000000000000000000000001E
:1002E000000000000000000000000000000000000E
:1002F00000000000000000000000000000000000FE
:1003000000000000000000000000000000000000ED
:1003100000000000000000000000000000000000DD
:1003200000000000000000000000000000000000CD
:1003300000000000000000000000000000000000BD
:1003400000000000000000000000000000000000AD
:10035000000000000000000000000000000000009D
:10036000000000000000000000000000000000008D
:10037000F9B30011000000000000000000000000C0
:10038000000000000000000000000000000000006D
:10039000000000000000000000000000000000005D
:1003A000000000000000000000000000951AFF1F80
:1003B000000000000000000000000000000000003D
:1003C000000000000000000000000000000000002D
:1003D000000000000000000000000000000000001D
:1003E000000000000000000000000000000000000D
:1003F00000000000000000000000000000000000FD
:08183800B070FF1F4118FF1FF3
:10184000024981F3088802F083FA0000B070FF1F9C
:1018500010B502F0A5FB072804D0122808D00228F2
:1018600008D010BD044A0420136B01331363F8E75A
:101870000220F6E71420F4E78466FF1FF8B507009E
:101880000C0026002500503630785135002804D150
:101890000300287058342370F8BD2978CA00481E08
:1018A0008141A3183800A25C5B68C9B2FFF7D0FF82
:1018B00000280DD12B78DA00A218013350602B706C
:1018C0003378044A013B3370136A01331362D8E75B
:1018D0000123DFE78466FF1F5C234343074910B5FC
:1018E000C9180B0058331B78012B05D1FFF7C6FF31
:1018F000034A936A0133936210BDC046B866FF1F66
:101900008466FF1F10B502F03BFA064A012113005E
:1019100010CB4942D967044B136002F0A1FB2000B1
:1019200010BDC04600E100E01000100010B504003A
:1019300002F026FA024B1C6002F092FB10BDC0467A
:1019400000E100E010B5040002F01AFA4021094A53
:10195000200013688B43136002F0CAFB01F064FDA2
:101960000022054B01201A60044B04321A6002F079
:10197000CFFBFEE71CF00040C4F00040C0F0004088
:10198000431E5A425341A022F0B5D2015B4213409C
:10199000154D164A40019B182A18127E8BB00191F2
:1019A000002A1BD01A000832D46F0022E6B206AF1C
:1019B000E4B294420EDC2818C369002B08D00199C8
:1019C00002AA117106AA049202AA167303A89847E4
:1019D0000BB0F0BD1978B9540132EAE71A7D1A78D4
:1019E00006AB01261A70E6E74469FF1F004000407D
:1019F000F0B5254B04004001C25C85B0002A2BD015
:101A00001A18117E002927D0917E002924D011793F
:101A1000022921D11689D788D168F51BADB22A1CBD
:101A2000102D00D9102292B2BE4217D118180123EE
:101A300003710023C269C38003819A4206D06846BD
:101A4000032103730171029301A890470820002C21
:101A500000D0192001F034FC05B0F0BD013C654216
:101A60006C41A0256442ED012C40084D1B186419FF
:101A7000074D0633013A92B2AA42EDD01888461CAF
:101A80001E80085C2070F5E74469FF1F004000409D
:101A9000FFFF00000F220E4B10B59868104002386F
:101AA0000A280BD802F0CEF80D0A0B0A0A110A0A0E
:101AB0000A0A060002210020FFF762FF10BD012183
:101AC000F9E70020FFF794FFF8E7DB6FF6E7C04681
:101AD000004000400F220E4B10B5986810400238AD
:101AE0000A280BD802F0AEF80E0A0B0A0A120A0AEC
:101AF0000A0A060002210120FFF742FF10BD012162
:101B00000800F9E70120FFF773FFF7E7DB6FF5E760
:101B10000090004013B5334C2378072B3DD8324B4F
:101B20001A78324B002A39D18022196852020A43AE
:101B30001A60252001F034FF20232D4A11680B4341
:101B4000802113606B460422C905086807331042E0
:101B500028D080210422C905C86810422ED08021D7
:101B60002020C905CA688243CA6014221A701A78F4
:101B7000002A2FD18021C905C86820320243CA60DB
:101B800014221A701A78002A28D11A4B1A7D22784A
:101B90005A601D221A705932DA6013BD1A6816494C
:101BA0000A40C5E7086802430A6014221A701A78CE
:101BB000002ACED01A78013AD2B2F7E7C8680243B9
:101BC000CA6014221A7019784A1ED2B21A700029FB
:101BD000F9D1C4E71A78013AD2B2C7E71A78013AC4
:101BE000D2B2CEE7B444FF1F7C45FF1F3CF000405B
:101BF000AC44FF1F00200040FFFFFEFF564B70B5B6
:101C00001B68012B03D1554A936D0133936502F094
:101C10002FFA534B534A1860534B544C1A6001230C
:101C2000534A1360534A13602378002B06D00622D0
:101C30005149524802F02CF900232370504A514B6D
:101C400010681B78C1B2002B0ED14F4CC0B2237864
:101C50005BB2002B4FDB237824785BB264B21B04A9
:101C600024021B191B1813600B1C50294ED950233A
:101C7000464A47491078DBB2FF2202284BD1086858
:101C8000444C454D267890432A78964254D9227880
:101C900024782E78023B5D10A31B6B435201D31AAC
:101CA00010335B111843086002F03AF9031F012B4F
:101CB00045D83A4B1B78002B06D0394B1B78002BAC
:101CC00002D0002002F0C4F8A122364B920099788D
:101CD000354B4A431B689B18832292009B181B7844
:101CE000033B012B03D8AF20400002F0F1F80122A2
:101CF0002E4BDA8270BD237824785BB264B2FF3356
:101D0000FF341B0424021B190138ABE7CAB2022AB4
:101D1000AED20223ACE70868254C264D26789043C6
:101D20002A78964208D9227824782D78023B5B10D5
:101D3000641B63435201B2E72378DBB2B2E70228A7
:101D4000D5D11D4B1B78013B022B03D91B4B1B78B4
:101D5000022BCCD16C20C8E79809FF1FFC0FFF1F96
:101D6000BC65FF1FFF3F000014100340C065FF1F4C
:101D70000C10034000100340D50BFF1F7211FF1F12
:101D8000B40003408C09FF1F680AFF1F490AFF1FA8
:101D900094000340460AFF1F470AFF1FF908FF1F70
:101DA0002209FF1F300DFF1F3409FF1FBC0BFF1F4F
:101DB000440AFF1F450AFF1F1C09FF1F2309FF1FBD
:101DC00010B502F0EDF90022014B1A8010BDC0469B
:101DD000B865FF1F10B502F0C3F9A121054A8900BB
:101DE0009478054A61431268044B5218528C1A8049
:101DF00010BDC046300DFF1F3409FF1FB865FF1F1F
:101E000010B50D4B0D4A9978A1239B004B431268E6
:101E1000D218531DD97F0A4B1B88994209D2441C02
:101E200007D0C82805D0D2695B1A5A43054B5343E3
:101E3000C01802F05DF810BD300DFF1F3409FF1F00
:101E4000B865FF1F7102000070B5244D2B68002B90
:101E500028D001F06DFF2B68D8402B680400002BC0
:101E600027D002F0BDF82B68D8401D4B1D4A997849
:101E7000A1239B004B431268D118D25C91239B0095
:101E8000002A20D0CA580132CA50174B17491B6884
:101E90000868834214D3D23B181A012A1AD0144B73
:101EA000186070BD01F044FF124B196802F0A8F8E9
:101EB000D3E702F095F80F4B196802F0A1F8D4E7C8
:101EC0000D495B18E8E7CA500C4B1B68DB68E41847
:101ED000201AE4E7F530FF30E1E7C0461C08FF1F99
:101EE000300DFF1F3409FF1F9C09FF1FBC65FF1F3A
:101EF000A009FF1F1808FF1F2DFF3F00C465FF1F2B
:101F000070B504000D00282916D10300A433C2883F
:101F10001B889B1A0B4A9BB293420DD906006A3666
:101F200005223100653001F0ABFE002804D13100FC
:101F3000200002F04DF870BD2900200002F028F9C1
:101F4000F9E7C046FE7F0000F8B50400012001F06B
:101F500027FF01F005FF174A1749106009680300C1
:101F60001648174E01601748776805680020AF4291
:101F700001D27068281A144D091928601348C162EB
:101F8000A421446A49032143416211490978002987
:101F900005D010490978022902D10F3B1360F8BD22
:101FA000012901D1083BF9E7032901D1053BF5E7F8
:101FB000033BF3E7E408FF1F28F00040340AFF1F4B
:101FC00028100040180AFF1F1C0AFF1F00F00040E5
:101FD0001C09FF1F4A0AFF1F70B580241025E40565
:101FE000A3682B43A36001F0F3FEA368AB43A36097
:101FF00070BD0000F7B5160080221C001023D2052A
:102000000191916805000B43936000225A4BD73031
:102010001A6001F09DFF9D232A002F009B00EB58C2
:10202000CA3201210092FC37002B01D00021009A16
:10203000386802F0BDF82900009BCB311A784F4B6D
:10204000D3351A604B780A781B0213438A7812043E
:102050001A43CB781B061343494A1BBA13604B79CA
:102060000A791B0213438A7912041A43CB7931008F
:102070001B061343434A1BBA13606B782A781B0272
:102080001343AA7812041A43EB781B0613433E4A03
:102090001BBA1360019A330213433C4A13603C4B52
:1020A00022001B1B9C4603293DDCB3089A00130049
:1020B0005142B21A032A46D1354AE018511A8278A1
:1020C0004078120400020243E05C043302430A60D9
:1020D0000022FF2B4BDDF0222E4B12011A600F2243
:1020E0002D4B1A602D4A1368002BFCD00023224A86
:1020F00027491360091B321D0B191B68043A180A83
:1021000023706070180C1B0EA070E3700434002A5A
:10211000F2DC802210213B68D20501333B609368DA
:102120008B439360F7BD6346D578981893782D0656
:102130001B042B43157804392B43557804322D02A8
:102140002B430360AFE7022A0AD1114AE05C511A1F
:10215000E2185278120202430A6004339BB2B7E7D6
:10216000012AB5D10A4A521AE15C1160F5E7084923
:1021700059180A600433ACE7000004403C000440F6
:102180003800044034000440300004400C00044097
:102190000001044004000440100004401400044006
:1021A000F7B5150080221C001023D205009191681C
:1021B00007000B4393600023654AD730136001F09A
:1021C000C7FE9D233E009B00F9583B00CA363200F3
:1021D000FC33002900D07FE0586801F0E9FF3900A6
:1021E00032785C4BCB311A604B780A781B02134370
:1021F0008A78AC4612041A43CB78281D1B06134379
:10220000554A1BBA13604B790A791B0213438A792A
:1022100012041A43CB791B061343504A1BBA1360AE
:102220004B7A0A7A1B0213438A7A12041A43CB7A36
:1022300021001B0613434A4A1BBA1360009A2B0263
:102240001343484A13602200474B1B1B0093009B1B
:10225000CE785B1801938B7836061B0433430E78D7
:10226000043833434E78043136023343019E3360E1
:102270000328ECDC0321A808431C9B0029408000B4
:1022800003292BD13849E5185E18A9786D78E35CED
:1022900009042D022943194331600300083300214A
:1022A000FF2B2DDD314B324919600F21314B196065
:1022B000012327490B60304B19680029FCD0062107
:1022C0001B680B40042B20D080220020D20593688D
:1022D0000A318B439360FEBD01217DE7022908D1BD
:1022E00021495D18E1184978E35C09021943296026
:1022F000D3E70129D3D11C495918E35C0B60CCE723
:102300001948181801600433CAE7002310490B600C
:102310006346002B0CDC3B00FC335A681021013271
:102320005A608022D205936801208B439360D2E7E4
:10233000009B9B181B68190A13705170190C1B0E17
:10234000D37004235B4291709C440432E0E7C046A2
:10235000000004403C0004403800044034000440C5
:10236000300004400C00044000010440040004401C
:10237000080F0000100004401400044070B5061E51
:1023800019D00222614B9B799343012B13D1604BEF
:102390001A78FF2A0FD15A78FF2A0CD19A78FF2A8F
:1023A00009D1DA78FF2A06D11A79FF2A03D15B799D
:1023B000FF2B00D1A7E0574B0C201A78012A08D038
:1023C0000022554D1A702B781A00093A042A01D8B8
:1023D000212070BD5A1F012AFAD94C4CA07B042839
:1023E00000D990E0A279032A00D98CE0821E012A4C
:1023F00003D862881F2A00D885E0002E61D0012E04
:1024000000D080E0A288012AE2D0002B0AD1013856
:10241000032803D801F016FC151D19151F202E7076
:1024200001F06EFE2B785A1E032A16D800253B4B6E
:102430001D602823237501F0DBFDA8422ED0A58066
:10244000C6E7022320202B70EAE7042322202B700A
:10245000E6E7032321202B70E2E7073B012BB7D8E7
:102460002F4B1B68DB6A9B06B2D52E4B1A78002ACD
:10247000AED1A27B911E012901D9002AA8D1022246
:1024800080211A702823284D89012878237501F0AE
:1024900027FD80212878890101F022FE0123A380F5
:1024A000224B1B78002B0AD0FA228021204B92006D
:1024B0001B8809025A431C4B187801F099FC002034
:1024C00087E701F05DFC2B78A680073B012B06D93E
:1024D00018482E7001F014FD1E2001F011FE114B62
:1024E000114C1A78002A06D0802100222078890118
:1024F0001A7001F0F5FC01F0B3FD8021207809028B
:1025000001F0EEFCDBE7122063E7C046A60BFF1FDD
:102510006B09FF1F1A09FF1F1C09FF1F4809FF1F36
:10252000C465FF1F2309FF1F1B09FF1F2109FF1F90
:102530002C09FF1F0010004010B5002901D001F048
:1025400017FC10BDF7B5604B01919978A1239B0052
:102550004B435E4A060014681022E418D6235B0041
:10256000E0583623FF33E35C00279343222B41D10D
:10257000574B0F3A1A600760012501F0A1FC019B3F
:102580001880E8235B00E35C002B01D0B34258DDE8
:102590000023504FFB70AD33FF33E3581A68002A15
:1025A00003D09B88DB439B071DD03823FF33E35CBC
:1025B000002B18D09B235B00E35C002B13D1D1339D
:1025C000FF33E35CB3420EDAA4235B00E15AE01868
:1025D000090A023101F024FD23000122FE33013EED
:1025E00001351A87FA70E8235B00E35C002B2AD0E0
:1025F000A8B2FEBD03683D00002BBED08188043028
:10260000090A023101F00CFDD6235B00E3581F607C
:10261000B2E72300B133BA00FF33985801378188FD
:102620000430090A023101F0FBFCE8235B00E35CA3
:10263000BB42EEDCE822F61AED1800235200A35448
:10264000A6E70027F1E7200001F012FB00281FD0C9
:10265000002E1DDD7319882647190193B60020004E
:1026600001F00EFD5A308000201840680135818845
:102670000430090A023101F0D3FC200001F088FB8C
:10268000A3590133A351BD4202D0019B9D42E6D123
:10269000114BE35C002BABD095239B00E35C002B3C
:1026A000A6D00E4BE15A0029A2D00D4AA35C994254
:1026B00002D90133A3549BE700231A212000A3541D
:1026C00001F0BEFB94E7C046300DFF1F3409FF1F29
:1026D00000140340E010FF1F5A02000072020000C5
:1026E0005E020000F8B51D4B1D4F1A78002A10D16C
:1026F000BA7B002A02D101321A7003E0032AFAD011
:10270000022AF8D001F074FC00220120154B1A7047
:10271000F8BD154B154D1C68154B9E7801232B7089
:102720002878C0B200F0DEFCBB7B002B0BD101F09F
:1027300047FCA1239B007343E41883239B00E41808
:1027400023782B70E4E7032B02D101F0F9FBF0E7CB
:102750000020022BDCD101F003FCEAE71C09FF1F7B
:10276000A60BFF1F2309FF1F3409FF1F490AFF1F84
:10277000300DFF1FF0B587B00EAD2F780FAD2D785F
:102780000593AC46634614000E4D0CAA12782E78C1
:1027900003930D9B009201932200059B029701F089
:1027A00087FA2E70012C01D0042C08D18022064912
:1027B0008B889343054A1278D20113438B8007B06C
:1027C000F0BDC0461C09FF1F6C11FF1F7809FF1FD9
:1027D0000B001B3B70B504003020E02B0DD813001C
:1027E000E025493BFF3B9BB2ED00AB4205D8034BD4
:1027F000200019825A8201F063FC70BD8410FF1F13
:1028000010B501F035FC054B00205B68052B04D9A1
:10281000034A5268D20200D4980810BD001000404C
:10282000FCE100E070B501F0ABFA0D4B1B68FC3326
:10283000DC691D6AFFF7E4FF6419844204D2094B86
:1028400001241B68002B07D004220024064B1A70B9
:10285000064A93690133936101F002FC200070BDC8
:10286000C465FF1F9809FF1F2309FF1FFC0FFF1FEF
:1028700070B50C4D2B68FC335C6A01F081FAFFF7F0
:10288000BFFF2B680025FC339B6AE318834204D208
:10289000054B1B68AB4200D1051B01F0E1FB280092
:1028A00070BDC046C465FF1F9809FF1FD722044BA7
:1028B00092009B5810B5002B00D0984710BDC04621
:1028C0000000FF1FF0B587B001F046F9FFF7EEFFFB
:1028D000CA4BCB4C04931B78022B45D1C94B1B68C8
:1028E000186A01F05DFAC84BC84A1A60C84BC94A59
:1028F0001A60A022C84B52001A60049B187801F09D
:1029000057FAC649C64801F003FBC649C64801F05C
:10291000FFFA1022C54BFF201A60802252031A6072
:10292000802292031A60802212041A6001F090FA49
:10293000012001F0DDF9FA20400001F0C9FB582028
:1029400001F0C6FABA4801F0E3F9012001F0B0FA4B
:10295000072001F055FA2268B64B1A4084235B0029
:102960001343236007B0F0BD01F012FBB24E02909A
:10297000322001F015FA33681B0629D43C2001F0FF
:102980000FFA0F2001F00CFA9C4B1B78012B00D1A1
:102990001EE180223368A94D134200D0A7E02B68C6
:1029A000032013432B6001F0FBF901F0F1FA029BC5
:1029B0000299C31A5A1E814200D81A00A04B1A600D
:1029C000904B19681E2353439E4A9B18CB618AE79C
:1029D00001F0DEFA80239C4ADB02116803900B436E
:1029E00013602268934B994F1A40282313432360A6
:1029F000032001F0D5F903203D6801F0D1F93B68CF
:102A00000320DB03DB0B009301F0CAF93B68ED0305
:102A1000DB03ED0BDB0B8E4A0193AB18C22B30D8D6
:102A2000009B9B18C22B2CD8019B9B18C22B28D82B
:102A3000009B2A009D4200D21A00009B9D4200D9B3
:102A40001D00019B934200D21300019A954200D9C8
:102A500015005B1B122B14D80C22336814209343EF
:102A6000336033687B4A1340336001F099F90821E1
:102A70003B682268DB038A432260774ADB0B1360E2
:102A80007FE7032001F08CF93B68DB03DB0B059348
:102A900001F07EFA039B0399C21A531E814200D8AB
:102AA00013006E4A93421BD9FF23356869492D0AEA
:102AB0001D4032686B1C1B060A401B0C134333601D
:102AC0000C23326800209A43083B1343336001F023
:102AD000DFF86348634BA840984206DCFEF732FFFC
:102AE000019B009D0093059B95E75F48F6E7002357
:102AF0005E4F554A3B6080231168DB020B43136035
:102B000080222B68032013432B6001F049F93B68B6
:102B1000052601333B6080232A685B0213432B6048
:102B20002268444B03201A40514B1343236001F0A9
:102B300037F90821454B1A682368D2038B43236079
:102B4000454B023900931B68D20B4B439A420CD879
:102B50009B1A3B2B0BD8236846490B4023602B68FC
:102B60000B402B60444B1A601FE7D31AF1E7013E7C
:102B7000F6B2002ED4D123683E4A134023602B685E
:102B800013402B603B68042B07D9BFF34F8F3B4B9F
:102B90003B4ADA60BFF34F8FFEE780222B680320A9
:102BA00093432B6001F0FCF82268224B03201A406B
:102BB00028231343236001F0F3F8244B009A1B6889
:102BC000DB03DB0B1360082223689343236097E742
:102BD00007222C4D2B681340012B02D1002001F05D
:102BE000E7F8AB68284A02201340AB6001F0D8F840
:102BF0008023AA685B001343AB60D6E64A0AFF1F36
:102C00005CF00040C465FF1F000003400180063DEA
:102C1000BC00034034080000A4000340710200001F
:102C200014100040FFFF3F002810004000E100E0CA
:102C30003075000000FEFEFFC4F0004044F000408C
:102C4000AC65FF1F7206000040F0004064F00040D9
:102C500091FCFFFFFF00FFFFB465FF1FE30C0000C6
:102C6000E88000005F361E0060361E001844FF1F1B
:102C700028000100FFFFFEFFB065FF1F00ED00E030
:102C80000400FA053CF00040FFFEFFFF694E336888
:102C900088331B6883F3088801F072F900F0C4FBE5
:102CA000654B664A1B68934207D0002000F0F0FF96
:102CB0000221634A13688B431360FFF703FE614BE5
:102CC000614C1878C0B201F053F90023A3600233BD
:102CD000A3605E4B0120236001F062F80323A36030
:102CE00001F056F9040001F0C3F9050001F050F9B4
:102CF000574B186001F09CF9564B1968621A531E25
:102D0000A14200D213008022D203934201D39B023E
:102D10009B0A3268D16AC90700D478E04E491C0C7E
:102D200009689BB24C4359432402090A64180327DB
:102D30004A49FC3293680A6849489B1A494A4A4EF4
:102D400012684A499B18414A34609A183B400193E3
:102D5000036892089C46019B0A6063440360042B4D
:102D600003D901323B400A6003600B684049E41814
:102D7000200001F045F93F4F3D493B68C3183B60D7
:102D80002000019301F0D4F93B4C20680818384921
:102D90002060884205D9019B01333B6001F0C8F9EE
:102DA000216000F08DFF354B1B78002B0ED001F019
:102DB0005FF93168324B4A1B1B6812189A4233D2B2
:102DC000591A4919091A2F4801F0A2F82E4C237AF2
:102DD000002B0FD001F04CF93168E3684A1B121840
:102DE000934224D9591A4919091A284801F090F830
:102DF00000232372264B83F3088801F049F902204F
:102E000001F07EF9002000F043FF00F0E9FFDC0153
:102E100099000234641A5900641A09214B43803323
:102E2000CB40A408E41882E7FA218900CBE71949CE
:102E3000DBE7C046C465FF1F0C0AFF1FB641210334
:102E400010000040490AFF1F14100040C409000090
:102E5000100AFF1F340AFF1F380AFF1F200AFF1F36
:102E6000280AFF1F1C0AFF1FA865FF1F240AFF1F57
:102E7000710200006008FF1F2C0AFF1F1C09FF1FC2
:102E8000E408FF1F00100040740BFF1F3C100040BF
:102E900000000020DC050000A022054B92009B589A
:102EA00010B5002B01D0984710BD00F0D9FFFBE70B
:102EB0000000FF1FA122054B92009B5810B5002B6C
:102EC00001D0984710BD00F0CBFFFBE70000FF1FCB
:102ED000A222054B92009B5810B5002B01D09847B9
:102EE00010BD00F0BDFFFBE70000FF1FA322054B54
:102EF00092009B5810B5002B01D0984710BD00F0F0
:102F0000AFFFFBE70000FF1FA422054B92009B5878
:102F100010B5002B01D0984710BD00F0A1FFFBE7D2
:102F20000000FF1F70B501F0A3F8514B186004209A
:102F300001F0E6F800F074FF0400C30702D400F0CB
:102F40009FFF70BD00224B4B1A604B4B1878013825
:102F500004282CD800F076FE03231B1F2700200036
:102F600000F0E6FF0128ECD0444C2378042B71D10B
:102F700000F096FF002806D001F01AF8582000F063
:102F8000A7FF02232370032001F0BAF8D9E720003D
:102F900000F0A6FEE6E7200001F0DAF8E2E7200004
:102FA00000F046FFDEE7200001F052F8DAE700F01B
:102FB000B7FF0500012808D1314B1B78053B012BD9
:102FC00003D82000FFF768FFCEE72C4B1B78022BBD
:102FD00001D0052B20D1022D28D12A4B9B7BAB435E
:102FE0001CD12000FFF766FF254B18780128BBD1C4
:102FF0006405B9D4234925224B7B034205D1233AEA
:1030000013405A42534126331A000B7D9342ABD9E9
:10301000322000F075FEA7E7022D07D1184B1B7870
:10302000052B11D12000FFF753FFDDE7012D0BD158
:10303000012B03D12000FFF759FF95E7062B03D1A1
:103040002000FFF761FF8FE7200000F009FF022D4D
:103050008AD1C9E7032B04D10B4B987C00F070FE9A
:1030600091E7072B8FD1094B987B01F019F88AE77C
:103070009C09FF1F9809FF1F9009FF1F2309FF1FCD
:103080001C09FF1FA60BFF1FBC0BFF1FD40BFF1F4C
:10309000FA210A4B0A4A49001A640A4A5A500A4A53
:1030A00004395A50094A08319A64094A5A50094A5F
:1030B0005C315A50084ADA667047C0460000FF1F6C
:1030C0007527FF1F7128FF1F2528FF1F7D23FF1F66
:1030D000E526FF1F011EFF1FD51DFF1F10B500F0C5
:1030E00099FD10BD8023F7B59C46264B264F0193D2
:1030F0002649274A274D284C284B02281AD16046DA
:1031000038600868264E3040802636033043086019
:1031100001990978002909D11660224A2A60224AB9
:103120002260E02219689143A03A1BE08021C90285
:103130001160F2E766463E600F68194E3E408027F8
:10314000FF023E430E600199097800290DD11760F6
:1031500001280ED1154A2A60154A2260E02219681A
:103160009143C03A0A431A60F7BD80218902116079
:10317000EEE7E0210F4A02432A600F4A22601A68F4
:103180008A43F0E74B0AFF1FE0000340D8000340EA
:103190009000034000000340500003404000034003
:1031A000FFFFE3FF0280063D804508220180063DC7
:1031B000806608220080069880550822F8B51E4BCC
:1031C00080261A68002014003440324232D11A6836
:1031D0001A4F32431A6001223B68063093433B602A
:1031E00000F0DEFD0122164D2B681E432E603B6869
:1031F0000A2613433B608027BF00124B1B683B42EB
:1032000011D1013EF6B2FF2E09D17E220E4B1C6871
:103210002B68E40B1440934323432B6005E0082004
:1032200000F0BEFDE9E7002EEFD180222B68600898
:1032300093432B60F8BDC046C4F000405CF00040F2
:1032400018F0004068F0004060F0004010B500F059
:10325000DFFD01215820034A00F022FDFFF7AEFFF9
:1032600010BDC046600AFF1F10B578220021034838
:1032700000F056FF00F054FD002010BDCC68FF1F89
:1032800070B5040000F07CFD00230C200B4A010007
:1032900059438D18515C00290DD0A14208D101235A
:1032A00000246B7000F06CFF00F0DAFE200070BDAF
:1032B00001330A2BEBD11224F6E7C046CC68FF1F7E
:1032C00070B5040000F05CFD002319001D000D4ADC
:1032D0001078002806D0A0420CD1557001310C3274
:1032E0000A29F5D1002B0AD100F01AFD00F0B8FE32
:1032F000002070BD5078461EB0411B18EEE700F06C
:103300003FFFF3E7CC68FF1FF7B504000C20002354
:1033100084460E4D019267465F43E85D7E19A042E8
:1033200012D000280BD10A4B9C4662461B7808330A
:103330001370019B70707C557160B360FEBD0133EA
:103340000A2BE8D10320F9E70720F7E7CC68FF1F35
:10335000C868FF1F8021204BC9051B6870B58B60B2
:103360001E4BC1241A680123FF2013434B611C4BE1
:10337000A4001A681B4B00251A601B4B1A681B4BD4
:103380001A601B4B1A5982431A51C52292009C584D
:103390008443BF38204398509C58164804408020EE
:1033A000C001204398509858134C0002000A014372
:1033B0009950124B1B78DB08AB4201DC002070BD3A
:1033C0002378002B06D0A368002B00D09847013546
:1033D0000C34EEE71220F2E7B044FF1FAC44FF1FAD
:1033E000B0F00040C468FF1FB4F00040C068FF1F89
:1033F00000E100E0FF00FFFFCC68FF1FC868FF1F6F
:10340000030010B51F2809D8072200201340072405
:1034100004490A78A24313430B7010BD0023062011
:10342000F5E7C046C868FF1F034A04491368002037
:103430000B4013607047C0461CF00040FFFFC1FF07
:10344000054B06491B780A6805485B0702401B0BC1
:10345000134300200B607047C868FF1F1CF000403A
:10346000FFFFC1FF70B50C25FFF7EAFF0A4B1C7880
:103470000A4BE4086543ED18002C01D1200070BD13
:103480002B78002B06D06B68002B00D09847013CAE
:103490000C3DF1E71220F2E7C868FF1FC068FF1F6C
:1034A00007B50422074801A900F034F9019B013354
:1034B00005D18023044ADB0411680B43136000200C
:1034C0000EBDC0461C18001114F00040F0B50500F8
:1034D0002026184B87B00493049B002B03D11124A2
:1034E000200007B0F0BD002102220B0001910091E5
:1034F000052000F025FE02230F490A681A42FCD17C
:103500000596059C631E0593002CFAD10B4A13689F
:10351000002BFCDA0F276F440121380000F090FDEA
:103520003B782B42DCD0052000F03AFC049B013BA9
:103530000493D1E7FFFFFF0790C8004000C8004098
:1035400007B500F01DFC80220821D205936A019185
:10355000002B01D10739916202210C4A11600199B7
:10356000481E01900029FAD1033111600531019103
:103570000199481E01900029FAD11160002B02D157
:103580008022D205936200F06BFD07BD00C00040B1
:10359000F0B52D4C89B02378002B4FD1FEF7B2F94E
:1035A00002232A4F03903A681A42FCD12023069343
:1035B000069B5A1E0692002BFAD1254E3368002B2B
:1035C000FCDA0120FFF782FF011E02D0112009B0B2
:1035D000F0BD030003220190009005AD9F2000F094
:1035E000AFFD0321280000F02BFD02233A681A42A8
:1035F000FCD120230793079B5A1E0792002BFAD178
:103600003368002BFCDA0120FFF760FF0028DDD1D2
:103610000398FEF78BF9AA786B7811041B020B4311
:1036200029780B4363601300113B0A49052B07D827
:1036300001239340A3600B60012323700020C6E7A1
:1036400080231B03F6E7C0469844FF1F90C8004044
:1036500000C800409808FF1F1E4B30B55A68187804
:103660001D4B85B0D31859424B41012100930023D3
:1036700000F07EFD194B1A4A02259A6300221A6552
:1036800010325A658022C4219D65164B1648D2021D
:10369000DA6789004258154B80241A4080231B04A6
:1036A00013434350642341200393E40500F078F969
:1036B000402000F075F96562039D6B1E0393002D99
:1036C000FAD103236362FFF73BFFA562FFF760FFB8
:1036D00005B030BDA444FF1F95FFFEF700C80040B1
:1036E000050001FF04E100E000E100E0FFFF00FF52
:1036F00010B5064B18705960FFF7AEFF002113207C
:10370000034AFFF701FE002010BDC046A444FF1F7E
:103710005936FF1FF0B5040085B003920291FEF701
:10372000F1F8882263035B0B52051A438023DB0503
:103730009D6A8023274F0092BA68002601901B03E0
:103740009A420CD9F82326001B041E401C4206D0C6
:103750008022214B52025E6219680A431A60002DD2
:103760000BD100F00DFB02221C4B1A608023DB05FD
:103770005A62013A9A6200F073FC0023039A934262
:1037800020D1002D0AD100F0FBFA144B03221D605A
:103790008023DB055A629D6200F062FC8023BA68D8
:1037A0001B039A4208D9002E06D000220A4B0C496E
:1037B0005A621A680A401A600198FEF7B7F80020AA
:1037C00005B0F0BD009A0299D2181278CA5401339C
:1037D000D4E7C0469844FF1F00C8004000C0004026
:1037E000FFFFFEFFF0B587B0029103920400FEF7E1
:1037F00089F8019000F0C4FA802302250122234EAB
:10380000DB0535605D629A6200F02AFC204F3B6860
:103810002B42FCD120230493049B5A1E0492002BBC
:10382000FAD11C4D2B68002BFCDA0120FFF74EFE6D
:10383000002802D0112007B0F0BD2000039A0299A1
:1038400000F046FA022304003A681A42FCD1202311
:103850000593059B5A1E0592002BFAD12B68002B6D
:10386000FCDA0120FFF732FE051EE3D100F088FAF2
:1038700080230322DB0535605A629D6200F0F0FB75
:103880000198FEF753F8E0B2D5E7C04600C000400B
:1038900090C8004000C80040F0B5802687B0040002
:1038A000FEF730F8F605B36A02250393029000F0A4
:1038B00067FA0123244F3D607562B36200F0D0FBCC
:1038C000224E33682B42FCD120230493049B5A1EC2
:1038D0000492002BFAD11E4D2B68002BFCDA01203C
:1038E000FFF7F4FD002802D0112007B0F0BD200042
:1038F00000F0BEFA0223019032681A42FCD1202364
:103900000593059B5A1E0592002BFAD12B68002BBC
:10391000FCDA0320FFF7DAFD041EE5D100F030FAEF
:1039200080230322DB053C605A629C6200F098FB16
:10393000039B002B01D1FFF703FE0298FDF7F6FF72
:103940006B461879D1E7C04600C0004090C80040DF
:1039500000C8004007B5000201910422000A01A935
:10396000FFF740FF0EBD000073B5050005240B4AAC
:10397000A3005B429B1819686B46DE1D300000F007
:1039800047FB022804D133782B55013CEFD276BD9A
:10399000052CFCD00128FAD10230F8E714090011F7
:1039A0001F2807D8012380228340D20591680B434A
:1039B000936070473F2808D8012380222038834035
:1039C000D20551690B435361F3E75F28F1D8012316
:1039D000802240388340D205116A0B431362E8E726
:1039E0001F2807D8012280218240C9058B68934394
:1039F0008B6070473F2808D8012280212038824000
:103A0000C9054B6993434B61F3E75F28F1D8012265
:103A1000802140388240C9050B6A93430B62E8E776
:103A20001F2810D880230200DB05153A1968012AE7
:103A300006D820229143196019680A431A6070471A
:103A400001228240F6E73F2811D880230200DB05DF
:103A5000353AD968032A06D810229143D960D9682B
:103A60000A43DA60EBE7012220388240F5E75F285D
:103A7000E5D842238022181A413B8340D205516A7F
:103A800099435162516A0B435362D8E710B5040061
:103A9000012813D1A022184992050B685B015B092C
:103AA00013430B60154B164A19681140154A0A4317
:103AB0001A60402219680A431A6010BD0028FCD120
:103AC00001000A2000F0F4FA21000B2000F0F0FAC7
:103AD000C0220A4B920019680A4340211A601A68F2
:103AE0008A431A60B022044912060B685B015B0925
:103AF00013430B60E1E7C04614F000401CF00040A7
:103B00007F00FEFF80FD010072B6074A1368013393
:103B100013600422054B1A600023054A13608022BB
:103B2000D2055360FEE7C0467808FF1FC0F0004092
:103B3000C4F00040044B054A1A60054B1A6000228D
:103B4000044B1A607047C046140AFF1F841E000011
:103B5000380AFF1FC4F000400023034A1360034AE1
:103B60001360034A1360704754F0004040F1004076
:103B700044F10040002310B5184C8AB00093019323
:103B80002378012B27D06946012000F019F900287D
:103B900017D1009B12490293019B06AA0393114B74
:103BA00002A81B680493104B1B68059300F010F9E2
:103BB00010220E4906A800F063F8002804D1FF2364
:103BC000237000200AB010BD0123094A074902A84A
:103BD000237000F0FDF80120F4E7C046C865FF1F20
:103BE00010290011082900110C29001120290011A9
:103BF000CC65FF1F13B501246946012000F0E0F8F1
:103C0000034B00940193FFF7B5FF200016BDC0469B
:103C1000BB0B000010B5FFF79FFFFFF7EBFF00287D
:103C200002D0024B984710BDFEE7C046E1A200005B
:103C300002B4714649084900095649008E4402BC45
:103C40007047C04602B4714649084900095C490002
:103C50008E4402BC7047C04603B471464908400018
:103C60004900095A49008E4403BC70470000000017
:103C700001B40248844601BC604700BF71B0000037
:103C800001B40248844601BC604700BFCD4C01002E
:103C900001B40248844601BC604700BF016C0100CA
:103CA00001B40248844601BC604700BF01670100BF
:103CB00001B40248844601BC604700BF9D6A000011
:103CC00001B40248844601BC604700BFD5440100EE
:103CD00001B40248844601BC604700BF95730100EF
:103CE00001B40248844601BC604700BF09340100AA
:103CF00001B40248844601BC604700BF691101005D
:103D000001B40248844601BC604700BF613701002E
:103D100001B40248844601BC604700BF8D11010018
:103D200001B40248844601BC604700BFADAE00004C
:103D300001B40248844601BC604700BFE90B0100A2
:103D400001B40248844601BC604700BF4DF9000041
:103D500001B40248844601BC604700BF05B40011AD
:103D600001B40248844601BC604700BFBD5C01004D
:103D700001B40248844601BC604700BFE9D400009A
:103D800001B40248844601BC604700BF75A9000029
:103D900001B40248844601BC604700BF5976010067
:103DA00001B40248844601BC604700BF018900009D
:103DB00001B40248844601BC604700BFEDA5000085
:103DC00001B40248844601BC604700BFE1AC00007A
:103DD00001B40248844601BC604700BFDD3F0000DB
:103DE00001B40248844601BC604700BF855201000F
:103DF00001B40248844601BC604700BF8B520100F9
:103E000001B40248844601BC604700BFF90D0100BF
:103E100001B40248844601BC604700BFED68010060
:103E200001B40248844601BC604700BFBD0B0100DD
:103E300001B40248844601BC604700BFF53501006B
:103E400001B40248844601BC604700BF53B900007A
:103E500001B40248844601BC604700BFED6B01001D
:103E600001B40248844601BC604700BFE917010065
:103E700001B40248844601BC604700BFA96F01003D
:103E800001B40248844601BC604700BFDD0A01005E
:103E900001B40248844601BC604700BFE94C010000
:103EA00001B40248844601BC604700BF01D700004E
:103EB00001B40248844601BC604700BFE51201001E
:103EC00001B40248844601BC604700BFCD0C01002C
:103ED00001B40248844601BC604700BF791201006A
:103EE00001B40248844601BC604700BFB3520100E0
:103EF00001B40248844601BC604700BF8937010015
:103F000001B40248844601BC604700BFC1A500005F
:103F100001B40248844601BC604700BF2D6C01001B
:103F200001B40248844601BC604700BFDD0C0100BB
:103F300001B40248844601BC604700BF013401005F
:103F400001B40248844601BC604700BF75F8000018
:103F500001B40248844601BC604700BF89440000A8
:103F600001B40248844601BC604700BF19FA000052
:103F700001B40248844601BC604700BF89140100B7
:103F800001B40248844601BC604700BFC9A90000D3
:103F900001B40248844601BC604700BF156B0100B4
:103FA00001B40248844601BC604700BFE927000015
:103FB00001B40248844601BC604700BF6DF60000B2
:103FC00001B40248844601BC604700BFE9F6000026
:103FD00001B40248844601BC604700BF85C10000AF
:103FE00001B40248844601BC604700BF6D0B01006C
:103FF00001B40248844601BC604700BFA9D8000054
:1040000001B40248844601BC604700BF090E0000AD
:1040100001B40248844601BC604700BF91380011DA
:1040200001B40248844601BC604700BFC1150100CD
:1040300001B40248844601BC604700BFC16601006C
:1040400001B40248844601BC604700BF3D710100D5
:1040500001B40248844601BC604700BFF935010045
:1040600001B40248844601BC604700BF9DA900001E
:1040700001B40248844601BC604700BFC95C01002E
:1040800001B40248844601BC604700BFD9B00000BB
:1040900001B40248844601BC604700BF7997000024
:1040A00001B40248844601BC604700BFC1F700006C
:1040B00001B40248844601BC604700BFF59F00116F
:1040C00001B40248844601BC604700BF116E000085
:1040D00001B40248844601BC604700BF851201005C
:1040E00001B40248844601BC604700BF0D52010084
:1040F00001B40248844601BC604700BFF9A6000035
:1041000001B40248844601BC604700BF19070100A2
:1041100001B40248844601BC604700BFA1AF000063
:1041200001B40248844601BC604700BFB70E0000DE
:1041300001B40248844601BC604700BF090E00007C
:1041400001B40248844601BC604700BF496D0100CC
:1041500001B40248844601BC604700BF0534010039
:1041600001B40248844601BC604700BFF9ED00007D
:1041700001B40248844601BC604700BFC56D010020
:1041800001B40248844601BC604700BF21A9000079
:1041900001B40248844601BC604700BF51B800002A
:1041A00001B40248844601BC604700BF8D82000014
:1041B00001B40248844601BC604700BF21440000AE
:1041C0000200000042BD001101000000F8BA001119
:1041D000020000003EBD0011010000000042FF1F70
:1041E0000200000000BB0011010000000863FF1F77
:1041F000020000003CBD0011030000007C62FF1FB4
:10420000120000000200000042BD00110100000089
:1042100040BB0011020000003EBD00110100000083
:104220003DBB0011020000004ABB0011030000006A
:10423000B762FF1F020000003CBD00110300000038
:10424000CC62FF1F020000003EBD00110100000013
:104250003CBB00110200000048BB0011030000003D
:104260008D62FF1F020000003CBD00110300000032
:10427000AE62FF1F0200000042BD001101000000FD
:1042800080BB0011020000003EBD001101000000D3
:104290004943FF1F0200000092BB00110100000013
:1042A0007BBB0011020000003EBD001101000000B8
:1042B0004843FF1F0200000090BB001101000000F6
:1042C000D462FF1F020000003EBD0011010000008B
:1042D0004743FF1F020000008EBB001101000000D9
:1042E0006BBB0011020000003EBD00110100000088
:1042F0004643FF1F020000008CBB001101000000BC
:1043000066BB0011020000003EBD0011010000006C
:104310004543FF1F020000008ABB0011010000009E
:1043200061BB0011020000003EBD00110100000051
:104330004443FF1F0200000088BB00110100000081
:104340005CBB00110202020202020000854A001159
:10435000834A0011D4BB0011900118001800FFFF20
:104360000701020304050602010600000000000028
:10437000000000000000000000000000000000003D
:1043800000000000000003000200000042BD001118
:104390000100000054BC0011020000003EBD0011ED
:1043A00001000000F843FF1F020000005EBC001186
:1043B000010000000263FF1F020000003CBD00116D
:1043C000030000007065FF1F020000003EBD0011E9
:1043D00001000000F843FF1F020000005CBC001158
:1043E000010000000463FF1F020000003CBD00113B
:1043F000030000006865FF1F12A6A6A600000000CB
:104400000001000000000111FFFF00005048593674
:10441000000000000000000001000000E5BB0011EA
:104420000B000500F7000000B40000280028002859
:104430003075A000A000A000A00000080008E00166
:10444000F0001000100010001000100010005000CC
:104450005000500010001000D007000000000000C5
:104460000F0001000500307507001000010081FFFA
:1044700000000000FF000000CD710011D56F001199
:10448000656D0011FFFF0100FF000000E99B0011B6
:10449000659900117D9800110000000000000000E7
:1044A00000000800040000003B0001085902E00180
:1044B00088212800FF0000000200000042BD00111A
:1044C0000100000008BE0011020000003EBD001106
:1044D000010000003545FF1F020000003ABD001139
:1044E000010000008469FF1F020000003EBD0011B2
:1044F000010000003445FF1F0200000038BD00111C
:10450000010000003245FF1F020000003EBD001107
:10451000010000003045FF1F0200000036BD001101
:10452000010000002845FF1F18001800000090013E
:1045300002000003020200000200000042BD001160
:10454000010000001CBE0011020000003EBD001171
:10455000010000007845FF1F0200000034BD00117B
:104560000000000000000000020000003CBD00113F
:0A45700003000000A469FF1F20FFF4
:040000051FFF184180
:00000001FF
